:020000040000FA
:0600000034EF45F0120090
:0A00060004000E8B0000C10400008E
:100010003A000000B18A0000210F0000010000003A
:10002000D18A0000840400003D000000B68A000070
:08003000E10000001B000000CC
:08003800D9CFE6FFDACFE6FFA5
:10004000E1CFD9FFE2CFDAFFE652E652FC0EDBCF7A
:10005000DEFFDBCFDDFFF80EDBCF00F0DB06F90EB5
:10006000DBCF01F001E2DB06005001100CE0DFCF36
:10007000E9FFDF2A010EDBCFEAFF01E3DB2AFA0EFC
:10008000DBCFEFFFE8D7E552E552E552E5CFDAFFE7
:10009000E7CFD9FF1200D9CFE6FFDACFE6FFE1CFF5
:1000A000D9FFE2CFDAFF060EE12402E3E168E6526F
:1000B000E16EFC0EDBCFDEFFDBCFDDFFFA0EDBCF28
:1000C0003FF0FB0EDBCF40F0020E3FC0DBFF030E24
:1000D00040C0DBFF040EDB6A050EDB6AF80EDBCFE7
:1000E00000F0DB06F90EDBCF01F001E2DB06005089
:1000F000011022E0DFCFE9FFDF2A010EDBCFEAFFAC
:1001000001E3DB2AEFCF04F0020EDBCFE9FFDB2AAD
:10011000030EDBCFEAFF01E3DB2AEF50045C026E43
:10012000036A02BE0368040E02C0DBFF050E03C0B3
:10013000DBFF02500310D2E0040EDBCF00F0050E0F
:10014000DBCF01F000C0F3FF01C0F4FF060EE15C5D
:1001500002E2E16AE552E16EE552E5CFDAFFE7CF70
:10016000D9FF1200D9CFE6FFDACFE6FFE1CFD9FF02
:10017000E2CFDAFF0C0EE12402E3E168E652E16E21
:100180000A0EFEC4DBFF0B0EFFC4DBFFD950FA0FD3
:10019000E96EFF0EDA20EA6E020EEE5C000EEE58FB
:1001A000000EEE58000EEE5801E27FD2FA0EDBCFC1
:1001B00000F0FB0EDBCF01F0FC0EDBCF02F0FD0EFA
:1001C000DBCF03F00A0EDBCFE9FF0B0EDBCFEAFF3C
:1001D000060EE926000EEA22EE50005CEE500158B1
:1001E000EE500258EE50035801E35FD20A0EDBCF07
:1001F000E9FF0B0EDBCFEAFFEF50030A01E1ACD1C0
:10020000010A01E146D1030A01E04FD2FA0EDBCF29
:100210003FF0FB0EDBCF40F0020E3FC0DBFF030ED2
:1002200040C0DBFF020EDBCF00F0030EDBCF01F09E
:10023000010E0F0B05E0D89001320032E806FBE119
:10024000D950020FE96E000EDA20EA6E0050EE2659
:100250000150ED22020EDBCF00F0030EDBCF01F0E8
:100260000001010E0116040E00C0DBFF050E01C0E7
:10027000DBFFD950020FE96E000EDA20EA6E090E9C
:100280000F0B06E0EC52D890ED32EF32E806FAE1BF
:10029000D950040FE96E000EDA20EA6EFF0EEE1858
:1002A00002E1010EED183FE0020EE66EE66A040E72
:1002B000DBCFE6FF050EDBCFE6FF020EDBCF00F063
:1002C000030EDBCF01F0026A036A0A0EDBCFE9FFFF
:1002D0000B0EDBCFEAFF0A0EE926000EEA22EE50F3
:1002E0000026EE500122EE500222EE50032200C002
:1002F000E6FF01C0E6FF02C0E6FF03C0E6FFD950FB
:10030000060FE66E000EDA20E66EBAEC3BF0046EE5
:100310000A0EE15C02E2E16AE552E16E0450000976
:1003200001E17FD0C2D1010EE66EE66AE668E66EB4
:10033000020EDBCF00F0030EDBCF01F0026A036A8E
:100340000A0EDBCFE9FF0B0EDBCFEAFF0A0EE92630
:10035000000EEA22EE500026EE500122EE5002225C
:10036000EE50032200C0E6FF01C0E6FF02C0E6FF38
:1003700003C0E6FFD950060FE66E000EDA20E66EE7
:10038000BAEC3BF0046E0A0EE15C02E2E16AE5526F
:10039000E16E0450000901E088D1010EE66EE66AC4
:1003A000000EE66EE66A020EDBCF04F0030EDBCF32
:1003B00005F0066A076A0A0EDBCFE9FF0B0EDBCFFA
:1003C000EAFF0A0EE926000EEA22EE500424006E2F
:1003D000EE500520016EEE500620026EEE50072012
:1003E000036E002A000E01220222032200C0E6FF53
:1003F00001C0E6FF02C0E6FF03C0E6FFD950070FC9
:10040000E66E000EDA20E66EBAEC3BF0086E0A0EDD
:10041000E15C02E2E16AE552E16E0850000901E0A8
:1004200044D1070EDBCF02F002C003F0026A060ED1
:10043000DB500210DE6E03C0DDFF010E046E056AA4
:10044000066A076AD950FA0FE96EFF0EDA20EA6EE3
:10045000EE500416EE500516EE500616EE50071636
:1004600004500510061007100BE0DECF00F0DDCFC2
:1004700001F0040ED89001320032E804FBE169D0AB
:10048000DECF00F0DDCF01F0FF0E00160F0E0116DB
:1004900060D0020EE66EE66AFA0EDBCF00F0FB0ECD
:1004A0000001016A010ED89000360136E806FBE132
:1004B00000C0E6FF01C0E6FFFA0EDBCF02F0FB0E44
:1004C000DBCF03F0FC0EDBCF04F0FD0EDBCF05F03D
:1004D000080ED8900532043203320232E806F9E100
:1004E0000A0EDBCFE9FF0B0EDBCFEAFF0A0EE9268F
:1004F000000EEA22EE500226EE500322EE500422B5
:10050000EE50052202C0E6FF03C0E6FF04C0E6FF8E
:1005100005C0E6FFD950060FE66E000EDA20E66E43
:10052000BAEC3BF0066E0A0EE15C02E2E16AE552CB
:10053000E16E0650000901E0B8D0070EDBCF04F0F1
:1005400004C005F0046A060EDB500410006E05C0FE
:1005500001F0026A036AA0D0040EE66EE66AFA0EA3
:10056000DBCF00F0FB0E0001016A009E020ED89066
:1005700000360136E806FBE100C0E6FF01C0E6FFF9
:10058000FA0EDBCF02F0FB0EDBCF03F0FC0EDBCF6D
:1005900004F0FD0EDBCF05F0070ED89005320432D3
:1005A00003320232E806F9E10A0EDBCFE9FF0B0E57
:1005B000DBCFEAFF0A0EE926000EEA22EE50022601
:1005C000EE500322EE500422EE50052202C0E6FF58
:1005D00003C0E6FF04C0E6FF05C0E6FFD950060FE2
:1005E000E66E000EDA20E66EBAEC3BF0066E0A0EFE
:1005F000E15C02E2E16AE552E16E0650000955E174
:10060000090EDBCF04F0056A066A076A180E1F0B95
:1006100007E0D8900436053606360736E806F9E1D5
:10062000080EDBCF08F0096A0A6A0B6A100E1F0B6E
:1006300007E0D890083609360A360B36E806F9E1A5
:1006400008500412095005120A5006120B500712E6
:10065000070EDBCF0CF00CC00DF00C6A0E6A0F6AAF
:100660000C5004120D5005120E5006120F500712B6
:10067000060EDBCF10F0116A126A136A04501010D4
:10068000006E05501110016E06501210026E0750D8
:100690001310036E0F0E031600C03DF001C03EF0B4
:1006A00002C03FF003C040F005D0010E3D6E3E6A2F
:1006B0003F6A406A0C0EE15C02E2E16AE552E16EDB
:1006C000E552E5CFDAFFE7CFD9FF1200D9CFE6FF39
:1006D000DACFE6FFE1CFD9FFE2CFDAFFE652E6520A
:1006E000FEC4DEFFFFC4DDFFD950FA0FE96EFF0E36
:1006F000DA20EA6E020EEE5E000EEE5AEE5AEE5A66
:10070000DECFE9FFDDCFEAFF060EE926000EEA2282
:10071000EECF00F0EECF01F0EECF02F0EFCF03F01E
:10072000020E005E000E015A025A035AD950FA0F07
:10073000E96EFF0EDA20EA6E0050EE5C0150EE58D2
:100740000250EE580350EE5805E33D6A3E6A3F6A98
:10075000406A46D0DECFE9FFDDCFEAFF120EE92680
:10076000000EEA22EECF08F0EECF09F0EECF0AF04D
:10077000EFCF0BF0DECFE9FFDDCFEAFF020EE92677
:10078000000EEA22EFCF04F0056A066A076A04C089
:100790003DF005C03EF006C03FF007C040F0FA0E45
:1007A000DBCF42F0FB0EDBCF43F0FC0EDBCF44F09F
:1007B000FD0EDBCF45F062EC44F039500824006EAA
:1007C0003A500920016E3B500A20026E3C500B202B
:1007D000036E00C03DF001C03EF002C03FF0406E2D
:1007E000E552E552E552E5CFDAFFE7CFD9FF120037
:1007F000D9CFE6FFDACFE6FFE1CFD9FFE2CFDAFFCC
:10080000060EE12402E3E168E652E16E040EFEC446
:10081000DBFF050EFFC4DBFFFC0EDBCFE9FFFD0EA7
:10082000DBCFEAFFEE6AED6AFC0EDBCFE9FFFD0EDF
:10083000DBCFEAFF040EE926000EEA22EECFDFFF4F
:10084000010EEECFDBFF020EEECFDBFF030EEECF8D
:10085000DBFFD9CFE9FFDACFEAFF010EEE1805E1A1
:10086000EE5003E1EE5001E1EE501FE0040EDBCF4D
:10087000E9FF050EDBCFEAFF060EE926000EEA22AD
:10088000EECF00F0EECF01F0EECF02F0EFCF03F0AD
:10089000D9CFE9FFDACFEAFF0050EE5C0150EE5805
:1008A0000250EE580350EE5802E3010E93D0D9CF18
:1008B000E9FFDACFEAFFEECF00F0EECF01F0EECFA6
:1008C00002F0EFCF03F000500110021003101EE100
:1008D000040EDBCFE9FF050EDBCFEAFFEF50030884
:1008E00015E1040EDBCFE9FF050EDBCFEAFF0E0EAC
:1008F000E926000EEA22EECFDFFF010EEECFDBFF8E
:10090000020EEECFDBFF030EEECFDBFFFC0EDBCFE4
:10091000E9FFFD0EDBCFEAFF080EE926000EEA2212
:10092000DFCFEEFF010EDBCFEEFF020EDBCFEEFFDF
:10093000030EDBCFEEFFD9CFE9FFDACFEAFFEECF30
:1009400004F0EECF05F0EECF06F0EFCF07F0045045
:100950000510061007101AE0D9CFE9FFDACFEAFF39
:10096000EECFE6FFEECFE6FFEECFE6FFEFCFE6FFFE
:10097000ADDEE552E552E552E5523DC000F03EC025
:1009800001F03FC002F040C003F012D0040EDBCFF4
:10099000E9FF050EDBCFEAFF0E0EE926000EEA2284
:1009A000EECF00F0EECF01F0EECF02F0EFCF03F08C
:1009B000FC0EDBCFE9FFFD0EDBCFEAFF0C0EE926D4
:1009C000000EEA2200C0EEFF01C0EEFF02C0EEFF03
:1009D00003C0EEFF006E060EE15C02E2E16AE55242
:1009E000E16E0050E552E5CFDAFFE7CFD9FF120004
:1009F000D9CFE6FFDACFE6FFE1CFD9FFE2CFDAFFCA
:100A0000080EE12402E3E168E652E16E060EFEC440
:100A1000DBFF070EFFC4DBFFFC0EDBCFE9FFFD0EA3
:100A2000DBCFEAFFEECF00F0EFCF01F0010E0026A2
:100A3000000E0122040E00C0DBFF050E01C0DBFF2B
:100A4000D950040FE96E000EDA20EA6EEE50ED1078
:100A500001E1D5D0FC0EDBCFE9FFFD0EDBCFEAFFD5
:100A60000C0EE926000EEA22EECF00F0EECF01F0E8
:100A7000EECF02F0EFCF03F0005001100210031090
:100A800001E1BDD0040EDBCF00F0050E016A0F0EB0
:100A900000160050011001E0F2D0FC0EDBCFE9FFA0
:100AA000FD0EDBCFEAFF0C0EE926000EEA22EE2A4D
:100AB000EE22EE22EE22FC0EDBCFE9FFFD0EDBCFB5
:100AC000EAFF080EE926000EEA22EECF00F0EECF94
:100AD00001F0EECF02F0EFCF03F000500110021052
:100AE00003101BE1040EDBCF00F0050EDBCF01F09D
:100AF000060EDBCFE9FF070EDBCFEAFF040EE92687
:100B0000000EEA22EECF02F0EFCF03F00250005CBD
:100B10000350015801E2B3D072D0040EDBCF02F0D3
:100B2000050EDBCF03F0040E0F0B05E0D890033267
:100B30000232E806FBE1060EDBCFE9FF070EDBCF52
:100B4000EAFF020EE926000EEA22EF040001021479
:100B5000006E016AE850011001E091D0FC0EDBCF7D
:100B6000E9FFFD0EDBCFEAFF080EE926000EEA22C0
:100B7000EECFE6FFEECFE6FFEECFE6FFEFCFE6FFEC
:100B8000B2EC00F0E552E552E552E5523DC0DEFF21
:100B90003EC0DEFF3FC0DEFF40C0DDFFDD52DD5264
:100BA000D9CFE9FFDACFEAFFD880010EEE54000E6C
:100BB000EE54000EEE54000EEE5402E3010E6CD023
:100BC000060EDBCFE9FF070EDBCFEAFF060EE926B4
:100BD000000EEA22EECF00F0EECF01F0EECF02F0F1
:100BE000EFCF03F0D9CFE9FFDACFEAFF0050EE5C98
:100BF0000150EE580250EE580350EE5802E3030E37
:100C00004BD0FC0EDBCFE9FFFD0EDBCFEAFF080E79
:100C1000E926000EEA22DFCFEEFF010EDBCFEEFF6A
:100C2000020EDBCFEEFF030EDBCFEEFFD9CFE9FFE5
:100C3000DACFEAFFEECFE6FFEECFE6FFEECFE6FF3C
:100C4000EFCFE6FF43DDE552E552E552E5523EC007
:100C500001F03FC002F040C003F0FC0EDBCFE9FF23
:100C6000FD0EDBCFEAFF0C0EE926000EEA223DC0A6
:100C7000EEFF01C0EEFF02C0EEFF03C0EEFFFC0E70
:100C8000DBCFE9FFFD0EDBCFEAFF040EDBCFEEFF8B
:100C9000050EDBCFEDFF000E006E080EE15C02E2F8
:100CA000E16AE552E16E0050E552E5CFDAFFE7CFA9
:100CB000D9FF1200D9CFE6FFDACFE6FFE1CFD9FFA7
:100CC000E2CFDAFFE652E652FC0EDBCFE6FFFD0E86
:100CD000DBCFE6FF8DDDE552E552DF6EDF5002E04F
:100CE000DF5098D0200EE66EE66AFC0EDBCFE9FFFF
:100CF000FD0EDBCFEAFFEECF00F0EFCF01F00001F9
:100D0000016A0F0E0016050ED89000360136E8066F
:100D1000FBE100C0E6FF01C0E6FFFC0EDBCFE9FF10
:100D2000FD0EDBCFEAFF0C0EE926000EEA22EECF25
:100D3000E6FFEECFE6FFEECFE6FFEFCFE6FFFA0EDF
:100D4000DBCFE6FFFB0EDBCFE6FFBAEC3BF0026E3B
:100D50000A0EE15C02E2E16AE552E16E025000092E
:100D600002E0010E01D0000EDF6EDF5052E1FA0EFC
:100D7000DBCFE9FFFB0EDBCFEAFF010EEFCFDBFF9E
:100D8000DB5003E1030EDF6E44D00B0EE76EFA0E6C
:100D9000DBCFE9FFFB0EDBCFEAFFE750E926000ED1
:100DA000EA22EF50080B28E10B0EE66EE66AFC0E15
:100DB000DBCFE9FFFD0EDBCFEAFF020EE926000ED6
:100DC000EA22EECFE6FFEFCFE6FFFA0EDBCFE6FF3B
:100DD000FB0EDBCFE6FF4BEC00F0026E060EE15C93
:100DE00002E2E16AE552E16E0250F3CF00F0F4CF87
:100DF00001F0F350F4100DE0FC0EDBCFE6FFFD0E2A
:100E0000DBCFE6FFF5DDE552E552DF6EDF5001E1B5
:100E100069D7DF50E552E552E552E5CFDAFFE7CF7B
:100E2000D9FF1200D9CFE6FFDACFE6FFE1CFD9FF35
:100E3000E2CFDAFF090EE12402E3E168E652E16E57
:100E4000FC0EDBCFE9FFFD0EDBCFEAFF020EE92649
:100E5000000EEA22050EEECFDBFF060EEDCFDBFF24
:100E60000B0EE66EE66A200EE66EE66A050EDBCF36
:100E7000E6FF060EDBCFE6FF1CEC00F0006E060E70
:100E8000E15C02E2E16AE552E16E0050040EDB6AC9
:100E9000030EDB6A080EF36E020EF3CFDBFFFA0ED1
:100EA000DBCFE9FFFB0EDBCFEAFF070EEECFDBFF68
:100EB000080EEDCFDBFF030EDBCFF3FFDB2AF35091
:100EC000E76E070EDBCFE9FF080EDBCFEAFFE75046
:100ED000E926000EEA22EFCFDFFFDF5020083CE2D8
:100EE0002F0EDF5C39E02E0EDF5C09E0020EDB50D6
:100EF000F36E040EDBCFF4FFF350F45C12E3020E4A
:100F0000DB50080829E12E0EDF5C26E1080EF36EA7
:100F1000040EF3CFDBFF0B0EF36E020EF3CFDBFFFD
:100F2000CAD7610EDF5C05E3DF507A0802E3200ECA
:100F3000DF5E040EDBCFF3FFDB2AF350E76E050E16
:100F4000DBCFE9FF060EDBCFEAFFE750E926000E14
:100F5000EA22DFCFEFFFAFD7030EDB50E76E070EBD
:100F6000DBCF00F0080EDBCF01F0E7500026000ECB
:100F70000122FA0EDBCFE9FFFB0EDBCFEAFF00C058
:100F8000EEFF01C0EDFFDF50200802E3010E01D0AB
:100F9000000EE66E0B0EE76E050EDBCFE9FF060EC8
:100FA000DBCFEAFFE750E926000EEA22E552E750E0
:100FB000EF6E000E006E090EE15C02E2E16AE5529E
:100FC000E16E0050E552E5CFDAFFE7CFD9FF12001E
:100FD000D9CFE6FFDACFE6FFE1CFD9FFE2CFDAFFE4
:100FE000E652F80EDBCFE9FFF90EDBCFEAFFEF5058
:100FF000200806E1F80EDB2AF90EF3E3DB2AF1D72D
:10100000F80EDBCFE9FFF90EDBCFEAFFEF502F0838
:1010100005E1F80EDB2AF90E01E3DB2AFC0EDBCF3B
:10102000E9FFFD0EDBCFEAFF040EE926000EEA22FF
:10103000EE6AEE6AEE6AEE6AF80EDBCFE9FFF90EB1
:10104000DBCFEAFFEF50200813E3FC0EDBCFE6FF17
:10105000FD0EDBCFE6FFF8EC03F0E552E552DF6E64
:10106000FA0EDBCFE9FFFB0EDBCFEAFFEF6AE0D041
:10107000D950F80FE66EFF0EDA20E66EFC0EDBCFDD
:10108000E6FFFD0EDBCFE6FFCDDEE552E552E55291
:10109000E552DF6EDF5001E0CBD0FA0EDBCFE6FF8A
:1010A000FB0EDBCFE6FFFC0EDBCFE6FFFD0EDBCF5A
:1010B000E6FF00DEE552E552E552E552DF6EDF5015
:1010C0001AE0030EDF5C01E0B3D0FC0EDBCFE9FFDA
:1010D000FD0EDBCFEAFF020EE926000EEA22EE50FB
:1010E000EFCFEAFFE96E0B0EE926000EEA22EF5081
:1010F00001E09ED024D0FC0EDBCFE9FFFD0EDBCF5C
:10110000EAFF020EE926000EEA22EE50EFCFEAFFD8
:10111000E96E0B0EE926000EEA22EF5001E088D0BE
:101120000B0EE76EFA0EDBCFE9FFFB0EDBCFEAFF1B
:10113000E750E926000EEA22EF50100B03E1040EFF
:10114000DF6E76D0140EE76EFA0EDBCFE9FFFB0EF2
:10115000DBCFEAFFE750E926000EEA22010EE9267E
:10116000000EEA22EFCF04F004C005F0046A140E6A
:10117000E76EFA0EDBCFE9FFFB0EDBCFEAFFE750AD
:10118000E926000EEA22EF500410006E05C001F0BF
:10119000026A036A100E1F0B07E0D8900036013672
:1011A00002360336E806F9E11A0EE76EFA0EDBCFD7
:1011B000E9FFFB0EDBCFEAFFE750E926000EEA224B
:1011C000010EE926000EEA22EFCF0AF00AC00BF06A
:1011D0000A6A1A0EE76EFA0EDBCFE9FFFB0EDBCFD1
:1011E000EAFFE750E926000EEA22EF5000010A105C
:1011F000066E0BC007F0086A096AE85000120B502F
:1012000001120850021209500312FC0EDBCFE9FF55
:10121000FD0EDBCFEAFF040EE926000EEA2200C035
:10122000EEFF01C0EEFF02C0EEFF03C0EEFF20D7CD
:10123000DF50E552E552E5CFDAFFE7CFD9FF1200E4
:10124000D9CFE6FFDACFE6FFE1CFD9FFE2CFDAFF71
:10125000020EE66EE66AFE0EE66E010EE66ED950EE
:10126000F80FE96EFF0EDA20EA6EEECFE6FFEECF62
:10127000E6FFEECFE6FFEFCFE6FFFC0EDBCFE6FFAB
:10128000FD0EDBCFE6FFBAEC3BF0006E0A0EE15C30
:1012900002E2E16AE552E16E0050000902E0030E4D
:1012A000BAD0010EE76EFC0EDBCFE9FFFD0EDBCFFF
:1012B000EAFFE750E926000EEA22EFCF02F002C073
:1012C00003F0026AFC0EDBCFE9FFFD0EDBCFEAFF85
:1012D000EF5000010210006E03C001F0550E00181F
:1012E00002E1AA0E011802E0020E95D0020EE66E8F
:1012F000E66A360EE66EE66AD950F80FE96EFF0E22
:10130000DA20EA6EEECFE6FFEECFE6FFEECFE6FFA5
:10131000EFCFE6FFFC0EDBCFE6FFFD0EDBCFE6FFF7
:10132000BAEC3BF0006E0A0EE15C02E2E16AE552C3
:10133000E16E0050000923E1010EE76EFC0EDBCFE9
:10134000E9FFFD0EDBCFEAFFE750E926000EEA22B7
:10135000EFCF03F003C004F0036AFC0EDBCFE9FF1C
:10136000FD0EDBCFEAFFEF5000010310016E04C059
:1013700002F0460E011803E1410E021849E0020E88
:10138000E66EE66A520EE66EE66AD950F80FE96E2E
:10139000FF0EDA20EA6EEECFE6FFEECFE6FFEECFED
:1013A000E6FFEFCFE6FFFC0EDBCFE6FFFD0EDBCF67
:1013B000E6FFBAEC3BF0006E0A0EE15C02E2E16A85
:1013C000E552E16E0050000925E1010EE76EFC0ECA
:1013D000DBCFE9FFFD0EDBCFEAFFE750E926000E89
:1013E000EA22EFCF03F003C004F0036AFC0EDBCF68
:1013F000E9FFFD0EDBCFEAFFEF5000010310016EA5
:1014000004C002F0460E011805E1410E021802E187
:10141000000E01D0010EE552E5CFDAFFE7CFD9FF8C
:101420001200D9CFE6FFDACFE6FFE1CFD9FFE2CF56
:10143000DAFF350EE12402E3E168E652E16E0401D1
:10144000FE6BFF6BD950FC0FE96EFF0EDA20EA6EDF
:10145000EE50ED1002E10EEF0FF04FEC3AF0010B01
:1014600003E0020E0FEF0FF0250EDB6A260EDB6A9B
:10147000270EDB6A280EDB6AD950250FE96E000EB5
:10148000DA20EA6EEECFE6FFEECFE6FFEECFE6FF24
:10149000EFCFE6FFD950010FE66E000EDA20E66EC0
:1014A000CFDE006E060EE15C02E2E16AE552E16E1B
:1014B0000050DF6EDF0401E09CD0100EE66EE66A9D
:1014C000BE0EE66E010EE66ED950250FE96E000ED7
:1014D000DA20EA6EEECFE6FFEECFE6FFEECFE6FFD4
:1014E000EFCFE6FFD950010FE66E000EDA20E66E70
:1014F000BAEC3BF0006E0A0EE15C02E2E16AE552F2
:10150000E16E0050000902E0030E72D0050EDB50C0
:1015100070E00C0EDBCF00F0016A026A036A180E5D
:101520001F0B07E0D8900036013602360336E80676
:10153000F9E10B0EDBCF04F0056A066A076A100EAC
:101540001F0B07E0D8900436053606360736E80646
:10155000F9E1045000120550011206500212075022
:1015600003120A0EDBCF08F008C009F0086A0A6A05
:101570000B6A08500012095001120A5002120B5057
:101580000312090EDBCF0CF00D6A0E6A0F6A0C50C5
:1015900000120D5001120E5002120F500312250EB0
:1015A00000C0DBFF260E01C0DBFF270E02C0DBFF01
:1015B000280E03C0DBFFD950250FE96E000EDA209C
:1015C000EA6EEECFE6FFEECFE6FFEECFE6FFEFCF1F
:1015D000E6FFD950010FE66E000EDA20E66E30DE2F
:1015E000006E060EE15C02E2E16AE552E16E005037
:1015F000DF6E030EDF5C2BE0DF5003E0070E0FEF22
:101600000FF0240EE66EE66A0D0EE66EE66AD9501D
:10161000250FE96E000EDA20EA6EEECFE6FFEECF80
:10162000E6FFEECFE6FFEFCFE6FFD950010FE66E03
:10163000000EDA20E66EBAEC3BF0006E0A0EE15CBA
:1016400002E2E16AE552E16E0050000902E0010E9B
:10165000E6D3D950170FE96E000EDA20EA6E0D0EB0
:10166000E95E000EEA5A010EE926000EEA22EFCFEB
:1016700002F002C003F0026AD950170FE96E000EA3
:10168000DA20EA6E0D0EE95E000EEA5AEF50000114
:101690000210006E290E00C0DBFF2A0E03C0DBFF24
:1016A0002B0EDB6A2C0EDB6A290EDBCF00F02A0E34
:1016B000DBCF01F02B0EDBCF02F02C0EDBCF03F0E3
:1016C000005001100210031001E082D0D950250F04
:1016D000E96E000EDA20EA6E0D0EE95E000EEA5A9F
:1016E000030EE926000EEA22EFCF00F0016A026A3B
:1016F000036A180E1F0B07E0D89000360136023639
:101700000336E806F9E1D950250FE96E000EDA201C
:10171000EA6E0D0EE95E000EEA5A020EE926000E90
:10172000EA22EFCF04F0056A066A076A100E1F0B63
:1017300007E0D8900436053606360736E806F9E1A4
:1017400004500012055001120650021207500312F5
:10175000D950250FE96E000EDA20EA6E0D0EE95E13
:10176000000EEA5A010EE926000EEA22EFCF08F039
:1017700008C009F0086A0A6A0B6A0850001209508A
:1017800001120A5002120B500312D950250FE96EB4
:10179000000EDA20EA6E0D0EE95E000EEA5AEFCF77
:1017A0000CF00D6A0E6A0F6A0C5000120D500112F7
:1017B0000E5002120F500312290E00C0DBFF2A0E3A
:1017C00001C0DBFF2B0E02C0DBFF2C0E03C0DBFFD2
:1017D000040EDBCF00F0016A026A036AD950290FB8
:1017E000E96E000EDA20EA6E00C042F001C043F05C
:1017F00002C044F003C045F0EECF3DF0EECF3EF026
:10180000EECF3FF0EFCF40F062EC44F03CC0EDFF94
:101810003BC0EDFF3AC0EDFF39C0EFFFD9500F0FCD
:10182000E96E000EDA20EA6E0D0EE95E000EEA5A4D
:10183000010EE926000EEA22EFCF04F004C005F005
:10184000046AD9500F0FE96E000EDA20EA6E0D0E11
:10185000E95E000EEA5AEF500410006E05C001F078
:10186000026A036AD950250FE96E000EDA20EA6E8B
:10187000EE500026EE500122EE500222EE500322DE
:10188000FC0EDBCFE9FFFD0EDBCFEAFF0A0EE926F7
:10189000000EEA2200C0EEFF01C0EEFF02C0EEFF24
:1018A00003C0EEFFFC0EDBCFE9FFFD0EDBCFEAFF4E
:1018B000020EE926000EEA22010EDBCFEFFFD9501F
:1018C000120FE96E000EDA20EA6E0D0EE95E000ED0
:1018D000EA5A010EE926000EEA22EFCF02F002C01A
:1018E00003F0026AD950120FE96E000EDA20EA6E98
:1018F0000D0EE95E000EEA5AEF500210006E03C0B2
:1019000001F0FC0EDBCFE9FFFD0EDBCFEAFF040E9A
:10191000E926000EEA2200C0EEFF01C0EDFFD9501B
:10192000140FE96E000EDA20EA6E0D0EE95E000E6D
:10193000EA5A010EE926000EEA22EFCF02F002C0B9
:1019400003F0026AD950140FE96E000EDA20EA6E35
:101950000D0EE95E000EEA5AEF500210006E2D0ED9
:1019600000C0DBFF2E0E03C0DBFF2F0EDB6A300E44
:10197000DB6A2D0EDBCF00F02E0EDBCF01F02F0E39
:10198000DBCF02F0300EDBCF03F00050011002106D
:10199000031001E082D0D950210FE96E000EDA2049
:1019A000EA6E0D0EE95E000EEA5A030EE926000EFD
:1019B000EA22EFCF00F0016A026A036A180E1F0BD9
:1019C00007E0D8900036013602360336E806F9E122
:1019D000D950210FE96E000EDA20EA6E0D0EE95E95
:1019E000000EEA5A020EE926000EEA22EFCF04F0BA
:1019F000056A066A076A100E1F0B07E0D8900436C6
:101A0000053606360736E806F9E10450001205509F
:101A100001120650021207500312D950210FE96E2D
:101A2000000EDA20EA6E0D0EE95E000EEA5A010E93
:101A3000E926000EEA22EFCF08F008C009F0086A94
:101A40000A6A0B6A08500012095001120A50021269
:101A50000B500312D950210FE96E000EDA20EA6E06
:101A60000D0EE95E000EEA5AEFCF0CF00D6A0E6A19
:101A70000F6A0C5000120D5001120E5002120F503E
:101A800003122D0E00C0DBFF2E0E01C0DBFF2F0E58
:101A900002C0DBFF300E03C0DBFFFC0EDBCFE9FF33
:101AA000FD0EDBCFEAFF020EE926000EEA22EFCFA1
:101AB0001AF01B6A1C6A1D6AD9500F0FE96E000EDE
:101AC000DA20EA6E0D0EE95E000EEA5A010EE926F2
:101AD000000EEA22EFCF14F014C015F0146AD950AA
:101AE0000F0FE96E000EDA20EA6E0D0EE95E000EB1
:101AF000EA5AEF5000011410106E15C011F0126A6E
:101B0000136AD9502D0FE96E000EDA20EA6E1050DC
:101B1000EE5C0C6E1550EE580D6E1250EE580E6EB7
:101B20001350EE580F6ED950290FE96E000EDA20CF
:101B3000EA6EEE500C5C086EEE500D58096EEE50D9
:101B40000E580A6EEE500F580B6EFC0EDBCFE9FFFD
:101B5000FD0EDBCFEAFF040EE926000EEA22EECFEF
:101B600016F0EFCF17F0040E0F0B05E0D8901732E8
:101B70001632E806FBE1186A196A1650085C046E12
:101B800017500958056E18500A58066E19500B5810
:101B9000076E04C03DF005C03EF006C03FF0406E49
:101BA0001AC042F01BC043F01CC044F01DC045F0F9
:101BB000C7EC44F03DC000F03EC001F03FC002F071
:101BC00040C003F0020E0026000E01220222032272
:101BD000310E00C0DBFF320E01C0DBFF330E02C04E
:101BE000DBFF340E03C0DBFFFC0EDBCFE9FFFD0E95
:101BF000DBCFEAFF060EE926000EEA22310EDBCF2C
:101C0000EEFF320EDBCFEEFF330EDBCFEEFF340EF6
:101C1000DBCFEEFF020EDF6ED950310FE96E000E02
:101C2000DA20EA6EF70EEE5C0F0EEE58000EEE585C
:101C3000000EEE5802E2010EDF6ED950310FE96E50
:101C4000000EDA20EA6EF70EEE5CFF0EEE58000E84
:101C5000EE58000EEE5802E3030EDF6EFC0EDBCFF3
:101C6000E9FFFD0EDBCFEAFFDFCFEFFF030EDF5C06
:101C700047E1230EDBCF00F0016A026A036A180E07
:101C80001F0B07E0D8900036013602360336E8060F
:101C9000F9E1220EDBCF04F0056A066A076A100E2E
:101CA0001F0B07E0D8900436053606360736E806DF
:101CB000F9E10450001205500112065002120750BB
:101CC0000312210EDBCF08F008C009F0086A0A6A87
:101CD0000B6A08500012095001120A5002120B50F0
:101CE0000312200EDBCF0CF00D6A0E6A0F6A0C5047
:101CF00000120D5001120E5002120F5003121ED08E
:101D0000290EDBCF00F02A0EDBCF01F02B0EDBCF4C
:101D100002F02C0EDBCF03F0FC0EDBCFE9FFFD0E53
:101D2000DBCFEAFF0A0EE926000EEA22EE5000267B
:101D3000EE500122EE500222EE500322FC0EDBCFC9
:101D4000E9FFFD0EDBCFEAFF0E0EE926000EEA22C8
:101D500000C0EEFF01C0EEFF02C0EEFF03C0EEFFC9
:101D6000290EDBCF00F02A0EDBCF01F02B0EDBCFEC
:101D700002F02C0EDBCF03F0FC0EDBCFE9FFFD0EF3
:101D8000DBCFEAFF0A0EE926000EEA22EE5000261B
:101D9000EE500122EE500222EE500322FC0EDBCF69
:101DA000E9FFFD0EDBCFEAFF040EE926000EEA2272
:101DB000EECF04F0EFCF05F0040E0F0B05E0D89046
:101DC00005320432E806FBE1066A076A0450002681
:101DD000055001220650022207500322FC0EDBCFE1
:101DE000E9FFFD0EDBCFEAFF120EE926000EEA2224
:101DF00000C0EEFF01C0EEFF02C0EEFF03C0EEFF29
:101E0000FC0EDBCFE9FFFD0EDBCFEAFFEE52EF6AFF
:101E1000FC0EDBCFFEF4FD0EDBCFFFF4000E006EF8
:101E2000350EE15C02E2E16AE552E16E0050E552F6
:101E3000E5CFDAFFE7CFD9FF1200D9CFE6FFDACF3F
:101E4000E6FFE1CFD9FFE2CFDAFF3F0EE12402E364
:101E5000E168E652E16E3D0EFEC4DBFF3E0EFFC4BC
:101E6000DBFFD9503D0FE96E000EDA20EA6EEE502E
:101E7000ED1002E1060EEBD03D0EDBCFE9FF3E0E8A
:101E8000DBCFEAFFEE52EF6AD950110F006E000E61
:101E9000DA20016E030E00C0DBFF040E01C0DBFF81
:101EA000FC0EDBCFE6FFFD0EDBCFE6FFD9501D0FAA
:101EB000E66E000EDA20E66ED950010FE66E000ED7
:101EC000DA20E66EE8EC07F0006E060EE15C02E256
:101ED000E16AE552E16E0050DF6EDF5002E0DF5054
:101EE000B6D01D0EDB5004E0280EDB50100B02E0D4
:101EF000030EADD0320EDBCF04F004C005F0046A4F
:101F0000310EDB500410006E05C001F0026A036A56
:101F1000100E1F0B07E0D89000360136023603364C
:101F2000E806F9E1380EDBCF0AF00AC00BF00A6AC6
:101F3000370EDB500A10086A096AE85000120B508D
:101F4000011208500212095003123D0EDBCFE9FFC7
:101F50003E0EDBCFEAFF1E0EE926000EEA2200C08D
:101F6000EEFF01C0EEFF02C0EEFF03C0EEFF3C0E2D
:101F7000DBCF00F0016A026A036A180E1F0B07E04C
:101F8000D8900036013602360336E806F9E13B0EFA
:101F9000DBCF04F0056A066A076A100E1F0B07E024
:101FA000D8900436053606360736E806F9E10450BF
:101FB00000120550011206500212075003123A0E89
:101FC000DBCF08F008C009F0086A0A6A0B6A0850FB
:101FD0000012095001120A5002120B500312390E5E
:101FE000DBCF0CF00D6A0E6A0F6A0C5000120D5018
:101FF00001120E5002120F5003123D0EDBCFE9FF0B
:102000003E0EDBCFEAFF1A0EE926000EEA2200C0E0
:10201000EEFF01C0EEFF02C0EEFF03C0EEFF3D0E7B
:10202000DBCFE9FF3E0EDBCFEAFF160EE926000EFE
:10203000EA22EE6AEE6AEE6AEE6A3D0EDBCFE9FF57
:102040003E0EDBCFEAFFEE52010EEF6E000E006E89
:102050003F0EE15C02E2E16AE552E16E0050E552BA
:10206000E5CFDAFFE7CFD9FF1200D9CFE6FFDACF0D
:10207000E6FFE1CFD9FFE2CFDAFF140EE12402E35D
:10208000E168E652E16EFC0EDBCF3FF0FD0EDBCFE8
:1020900040F0100E3FC0DBFF110E40C0DBFF120E00
:1020A000FEC4DBFF130EFFC4DBFFF80EDBCFE9FF3E
:1020B000F90EDBCFEAFFEE6AED6AD950120FE96E36
:1020C000000EDA20EA6EEE50ED1002E1060E87D225
:1020D000120EDBCFE9FF130EDBCFEAFFEE52EF501B
:1020E000010B02E1050E7BD2120EDBCFE9FF130ECE
:1020F000DBCFEAFF1A0EE926000EEA22EECF04F04B
:10210000EECF05F0EECF06F0EFCF07F0120EDBCFEB
:10211000E9FF130EDBCFEAFF160EE926000EEA22D6
:10212000EE50045C006EEE500558016EEE500658FD
:10213000026EEE500758036E090E00C0DBFF0A0E58
:1021400001C0DBFF0B0E02C0DBFF0C0E03C0DBFF88
:10215000FA0EDBCF00F0FB0EDBCF01F0026A036A60
:10216000D950090FE96E000EDA20EA6E0050EE5CDD
:102170000150EE580250EE580350EE580CE2090E92
:10218000DBCF3FF00A0EDBCF40F0FA0E3FC0DBFFA3
:10219000FB0E40C0DBFFD950FA0FE96EFF0EDA20CC
:1021A000EA6EEE50ED1001E10FD2120EDBCFE9FF27
:1021B000130EDBCFEAFF160EE926000EEA22EECF61
:1021C00000F0EECF01F0010E0116026A036A005022
:1021D00001100210031001E010D1120EDBCFE9FF55
:1021E000130EDBCFEAFF160EE926000EEA22EECF31
:1021F00000F0EECF01F0EECF02F0EFCF03F0090ECA
:10220000D8900332023201320032E806F9E1120EB0
:10221000DBCFE9FF130EDBCFEAFF020EE926000E4B
:10222000EA22EF04046E056A066A076AE85000169F
:102230000550011606500216075003160F0E00C077
:10224000DBFFDB5001E07DD0120EDBCFE9FF130E88
:10225000DBCFEAFF160EE926000EEA22EECF04F0ED
:10226000EECF05F0EECF06F0EFCF07F004500510EB
:102270000610071013E1120EDBCFE9FF130EDBCFC0
:10228000EAFF1E0EE926000EEA22EECF00F0EECFA6
:1022900001F0EECF02F0EFCF03F020D0120EDBCF33
:1022A000E9FF130EDBCFEAFF220EE926000EEA2239
:1022B000EECFE6FFEECFE6FFEECFE6FFEFCFE6FF95
:1022C000B2EC00F0E552E552E552E5523DC000F0B7
:1022D0003EC001F03FC002F040C003F0010E00C05C
:1022E000DBFF020E01C0DBFF030E02C0DBFF040EAA
:1022F00003C0DBFFD950010FE96E000EDA20EA6E51
:10230000D880010EEE54000EEE54000EEE54000E76
:10231000EE5401E35BD1120EDBCFE9FF130EDBCFEE
:10232000EAFF220EE926000EEA22010EDBCFEEFFC5
:10233000020EDBCFEEFF030EDBCFEEFF040EDBCF92
:10234000EEFF120EDBCFE9FF130EDBCFEAFF220E0A
:10235000E926000EEA22EECFE6FFEECFE6FFEECF53
:10236000E6FFEFCFE6FF66EC03F0E552E552E552FB
:10237000E552050E3DC0DBFF060E3EC0DBFF070E3B
:102380003FC0DBFF080E40C0DBFF050EDBCF00F0D7
:10239000060EDBCF01F0070EDBCF02F0080EDBCF1D
:1023A00003F0005001100210031001E10FD10F0ED5
:1023B000DBCF00F0016A026A036AD950050FE96EAB
:1023C000000EDA20EA6EEE500026EE500122EE50AA
:1023D0000222EE500322120EDBCFE9FF130EDBCFF9
:1023E000EAFF260EE926000EEA2200C0EEFF01C039
:1023F000EEFF02C0EEFF03C0EEFF046A020E056EA0
:10240000066A076A120EDBCFE9FF130EDBCFEAFF85
:10241000160EE926000EEA22EECF3DF0EECF3EF09A
:10242000EECF3FF0EFCF40F0426A020E436E446AB7
:10243000456AC7EC44F03950045C006E3A500558C8
:10244000016E3B5006583C5007580D0E00C0DBFF94
:102450000E0E01C0DBFF0D0EDBCF00F00E0EDBCF4A
:1024600001F0FA0EDBCF02F0FB0EDBCF03F00050E1
:10247000025C015003580CE2FA0EDBCF3FF0FB0E7A
:10248000DBCF40F00D0E3FC0DBFF0E0E40C0DBFF88
:102490000D0EDBCFE6FF0E0EDBCFE6FF120EDBCF1D
:1024A000E9FF130EDBCFEAFF160EE926000EEA2243
:1024B000EECF00F0EECF01F0010E0116026A036AC2
:1024C00000C0E6FF01C0E6FF120EDBCFE9FF130EEE
:1024D000DBCFEAFF260EE926000EEA22EECFE6FF6A
:1024E000EECFE6FFEECFE6FFEFCFE6FFD950FC0FD1
:1024F000E96EFF0EDA20EA6EEE50ED1003E1046A99
:10250000056A06D0100EDBCF04F0110EDBCF05F00C
:1025100004C0E6FF05C0E6FFBAEC3BF0066E0A0E0B
:10252000E15C02E2E16AE552E16E0650DF6EDF50E7
:102530004DE10D0EDBCF00F00E0EDBCF01F0026A95
:10254000036A120EDBCFE9FF130EDBCFEAFF160E94
:10255000E926000EEA220050EE260150EE2202503B
:10256000EE220350EE220D0EDBCF00F00E0EDBCF7D
:1025700001F0D950100FE96E000EDA20EA6E00501B
:10258000EE260150ED220D0EDBCF00F00E0EDBCF5C
:1025900001F0D950FA0FE96EFF0EDA20EA6E005012
:1025A000EE5E0150ED5A0D0EDBCF00F00E0EDBCFCC
:1025B00001F0F80EDBCFE9FFF90EDBCFEAFF0050A8
:1025C000EE260150ED22E7D5000E09D0120EDBCF2A
:1025D000E9FF130EDBCFEAFFEE52EF6A010E006E49
:1025E000140EE15C02E2E16AE552E16E0050E55250
:1025F000E5CFDAFFE7CFD9FF1200D9CFE6FFDACF78
:10260000E6FFE1CFD9FFE2CFDAFF130EE12402E3C8
:10261000E168E652E16EFC0EDBCF3FF0FD0EDBCF52
:1026200040F00C0E3FC0DBFF0D0E40C0DBFF110E73
:10263000FEC4DBFF120EFFC4DBFFF80EDBCFE9FFA9
:10264000F90EDBCFEAFFEE6AED6AD950110FE96EA1
:10265000000EDA20EA6EEE50ED1002E1060EDFD237
:10266000110EDBCFE9FF120EDBCFEAFFEE52EF5087
:10267000010B02E1050ED3D2D950FA0FE96EFF0E1D
:10268000DA20EA6EEE50ED1027E1110EDBCFE9FF04
:10269000120EDBCFEAFFEE52EF50400B14E0E66A79
:1026A000E66AE66AE66A000EE66EE66A8BEC3CF0E5
:1026B000006E060EE15C02E2E16AE552E16E005056
:1026C000000901E0A3D2110EDBCFE9FF120EDBCF30
:1026D000EAFFEE52EF9C98D2110EDBCFE9FF120E0B
:1026E000DBCFEAFFEE52EF50400B0CE1110EDBCFD7
:1026F000E9FF120EDBCFEAFF160EE926000EEA22F2
:10270000EE6AEE90110EDBCFE9FF120EDBCFEAFF8F
:102710001A0EE926000EEA22EECF04F0EECF05F005
:10272000EECF06F0EFCF07F0110EDBCFE9FF120E70
:10273000DBCFEAFF160EE926000EEA22EE50045C1B
:10274000006EEE500558016EEE500658026EEE50C7
:102750000758036E080E00C0DBFF090E01C0DBFF47
:102760000A0E02C0DBFF0B0E03C0DBFFFA0EDBCF4D
:1027700000F0FB0EDBCF01F0026A036AD950080FAC
:10278000E96E000EDA20EA6E0050EE5C0150EE5861
:102790000250EE580350EE580CE2080EDBCF3FF02B
:1027A000090EDBCF40F0FA0E3FC0DBFFFB0E40C04E
:1027B000DBFFD950FA0FE96EFF0EDA20EA6EEE5019
:1027C000ED1001E121D2110EDBCFE9FF120EDBCFBC
:1027D000EAFF160EE926000EEA22EECF00F0EFCF58
:1027E00001F00001010E01160050011001E035D189
:1027F000110EDBCFE9FF120EDBCFEAFF160EE92642
:10280000000EEA22EECF00F0EECF01F0EECF02F0A4
:10281000EFCF03F0090ED8900332023201320032BA
:10282000E806F9E1110EDBCFE9FF120EDBCFEAFF7C
:10283000020EE926000EEA22EF04046E056A066A1B
:10284000076AE85000160550011606500216075098
:1028500003160E0E00C0DBFFDB5001E079D0110E35
:10286000DBCFE9FF120EDBCFEAFF160EE926000EE2
:10287000EA22EECF04F0EECF05F0EECF06F0EFCF78
:1028800007F0045005100610071013E1110EDBCFFE
:10289000E9FF120EDBCFEAFF1E0EE926000EEA2248
:1028A000EECF00F0EECF01F0EECF02F0EFCF03F06D
:1028B00020D0110EDBCFE9FF120EDBCFEAFF220E94
:1028C000E926000EEA22EECFE6FFEECFE6FFEECFDE
:1028D000E6FFEFCFE6FFB2EC00F0E552E552E5523D
:1028E000E5523DC000F03EC001F03FC002F040C0E4
:1028F00003F000C0DFFF010E01C0DBFF020E02C0CB
:10290000DBFF030E03C0DBFFD9CFE9FFDACFEAFF1D
:10291000D880010EEE54000EEE54000EEE54000E60
:10292000EE5401E373D1110EDBCFE9FF120EDBCFC2
:10293000EAFF220EE926000EEA22DFCFEEFF010EAB
:10294000DBCFEEFF020EDBCFEEFF030EDBCFEEFFA1
:10295000110EDBCFE9FF120EDBCFEAFF220EE926D4
:10296000000EEA22EECFE6FFEECFE6FFEECFE6FF67
:10297000EFCFE6FF66EC03F0E552E552E552E55293
:10298000040E3DC0DBFF050E3EC0DBFF060E3FC060
:10299000DBFF070E40C0DBFF040EDBCF00F0050EAF
:1029A000DBCF01F0060EDBCF02F0070EDBCF03F02A
:1029B000005001100210031001E128D10E0EDBCFF0
:1029C00000F0016A026A036AD950040FE96E000E32
:1029D000DA20EA6EEE500026EE500122EE5002227E
:1029E000EE500322110EDBCFE9FF120EDBCFEAFF20
:1029F000260EE926000EEA2200C0EEFF01C0EEFF1F
:102A000002C0EEFF03C0EEFF110EDBCFE9FF120E96
:102A1000DBCFEAFF260EE926000EEA22EECFE6FF24
:102A2000EECFE6FFEECFE6FFEFCFE6FFE66EE66A1B
:102A30008BEC3CF0006E060EE15C02E2E16AE552CE
:102A4000E16E0050000901E0E1D0110EDBCFE9FF9B
:102A5000120EDBCFEAFFEE52EF8C110EDBCFE9FF57
:102A6000120EDBCFEAFF160EE926000EEA22EECFA9
:102A700000F0EFCF01F00001010E0116000ED8802A
:102A80000056020E01560F0E00C0DBFF100E01C0F3
:102A9000DBFF0F0EDBCF00F0100EDBCF01F0FA0EE4
:102AA000DBCF02F0FB0EDBCF03F00050025C0150E5
:102AB00003580CE2FA0EDBCF3FF0FB0EDBCF40F009
:102AC0000F0E3FC0DBFF100E40C0DBFF0F0EDBCF51
:102AD00000F0100EDBCF01F0026A036A00C0E6FFCF
:102AE00001C0E6FF02C0E6FF03C0E6FF0C0EDBCF2D
:102AF000E6FF0D0EDBCFE6FF8BEC3CF0046E060E1E
:102B0000E15C02E2E16AE552E16E0450000901E095
:102B10007DD00F0EDBCF00F0100EDBCF01F0026A8C
:102B2000036A110EDBCFE9FF120EDBCFEAFF160EB0
:102B3000E926000EEA220050EE260150EE22025055
:102B4000EE220350EE220F0EDBCF00F0100EDBCF93
:102B500001F0D9500C0FE96E000EDA20EA6E005039
:102B6000EE260150ED220F0EDBCF00F0100EDBCF72
:102B700001F0D950FA0FE96EFF0EDA20EA6E00502C
:102B8000EE5E0150ED5A0F0EDBCF00F0100EDBCFE2
:102B900001F0F80EDBCFE9FFF90EDBCFEAFF0050C2
:102BA000EE260150ED22110EDBCFE9FF120EDBCF36
:102BB000EAFF160EE926000EEA22EECF00F0EFCF74
:102BC00001F00001010E01160050011001E0F1D5E5
:102BD000E66AE66AE66AE66A000EE66EE66A8BEC8C
:102BE0003CF0006E060EE15C02E2E16AE552E16E45
:102BF000005000090BE1110EDBCFE9FF120EDBCF15
:102C0000EAFFEE52EF9CD5D5000E09D0110EDBCFB6
:102C1000E9FF120EDBCFEAFFEE52EF6A010E006E03
:102C2000130EE15C02E2E16AE552E16E0050E5520A
:102C3000E5CFDAFFE7CFD9FF1200D9CFE6FFDACF31
:102C4000E6FFE1CFD9FFE2CFDAFF120EE12402E383
:102C5000E168E652E16E100EFEC4DBFF110EFFC408
:102C6000DBFFD950100FE96E000EDA20EA6EEE504D
:102C7000ED1002E1060EEDD2100EDBCFE9FF110ED2
:102C8000DBCFEAFFEE52EF50010B02E1050EE1D27D
:102C9000FA0EDBCF00F0FB0EDBCF01F0FC0EDBCF3A
:102CA00002F0FD0EDBCF03F0100EDBCFE9FF110EBB
:102CB000DBCFEAFF1A0EE926000EEA220050EE5C96
:102CC0000150EE580250EE580350EE5816E2100E26
:102CD000DBCFE9FF110EDBCFEAFF1A0EE926000E6B
:102CE000EA22FA0EEECFDBFFFB0EEECFDBFFFC0E8F
:102CF000EECFDBFFFD0EEECFDBFF100EDBCFE9FFEB
:102D0000110EDBCFEAFF160EE926000EEA220C0EAA
:102D1000EECFDBFF0D0EEECFDBFF0E0EEECFDBFFB7
:102D20000F0EEECFDBFF100EDBCFE9FF110EDBCF76
:102D3000EAFF160EE926000EEA22EE6AEE6AEE6A55
:102D4000EE6AD950FA0FE96EFF0EDA20EA6ED880EB
:102D5000000EEE54000EEE54000EEE54000EEE5433
:102D600001E36CD2100EDBCFE9FF110EDBCFEAFFDF
:102D7000020EE926000EEA22EFCF3DF03E6A3F6ADE
:102D8000406A426A020E436E446A456A62EC44F04D
:102D9000040E39C0DBFF050E3AC0DBFF060E3BC058
:102DA000DBFF070E3CC0DBFFD9500C0FE96E000EB5
:102DB000DA20EA6ED880000EEE54000EEE54000EBB
:102DC000EE54000EEE5401E3D5D00C0EDBCF08F02C
:102DD0000D0EDBCF09F00E0EDBCF0AF00F0EDBCFAE
:102DE0000BF00806000E095A0A5A0B5A08C03DF0AB
:102DF00009C03EF00AC03FF00BC040F0040EDBCF2C
:102E000042F0050EDBCF43F0060EDBCF44F0070E99
:102E1000DBCF45F0C7EC44F03DC004F03EC005F008
:102E20003FC006F040C007F0FA0EDBCF00F0FB0E0B
:102E3000DBCF01F0FC0EDBCF02F0FD0EDBCF03F0A9
:102E40000006000E015A025A035A00C03DF001C0AC
:102E50003EF002C03FF003C040F0040EDBCF42F072
:102E6000050EDBCF43F0060EDBCF44F0070EDBCFC1
:102E700045F0C7EC44F004503D5C05503E58065008
:102E80003F580750405876E30C0EDBCF00F00D0E94
:102E9000DBCF01F00E0EDBCF02F00F0EDBCF03F025
:102EA0000006000E015A025A035A040EDBCF04F04A
:102EB000050EDBCF05F0060EDBCF06F0070EDBCFED
:102EC00007F00406000E055A065A075A041E051E8E
:102ED000061E071E04500016055001160650021665
:102EE00007500316100EDBCFE9FF110EDBCFEAFF10
:102EF000160EE926000EEA2200C0EEFF01C0EEFF2A
:102F000002C0EEFF03C0EEFF100EDBCFE9FF110E93
:102F1000DBCFEAFF160EE926000EEA22EECF00F024
:102F2000EECF01F0EECF02F0EFCF03F0D950FA0F61
:102F3000E96EFF0EDA20EA6E0050EE5E0150EE5AA6
:102F40000250EE5A0350EE5A100EDBCFE9FF110E7D
:102F5000DBCFEAFF220EE926000EEA22EECFDFFFEA
:102F6000010EEECFDBFF020EEECFDBFF030EEECF46
:102F7000DBFF2AD0100EDBCFE9FF110EDBCFEAFF1B
:102F80001E0EE926000EEA22EECFDFFF010EEECF85
:102F9000DBFF020EEECFDBFF030EEECFDBFF100EEA
:102FA000DBCFE9FF110EDBCFEAFF220EE926000E90
:102FB000EA22DFCFEEFF010EDBCFEEFF020EDBCF0A
:102FC000EEFF030EDBCFEEFF040EDBCF00F0050EAD
:102FD000DBCF01F0060EDBCF02F0070EDBCF03F0F4
:102FE000D950FA0FE96EFF0EDA20EA6EEE50005C5F
:102FF000EE500158EE500258EE50035801E389D0CC
:10300000D9CFE9FFDACFEAFFEECFE6FFEECFE6FF5A
:10301000EECFE6FFEFCFE6FFB2EC00F0E552E5526F
:10302000E552E5523DC0DEFF3EC0DEFF3FC0DEFFA1
:1030300040C0DDFFDD52DD52D9CFE9FFDACFEAFF34
:10304000D880010EEE54000EEE54000EEE54000E29
:10305000EE5401E3F5D0100EDBCFE9FF110EDBCF0C
:10306000EAFF060EE926000EEA22EECF00F0EECFD0
:1030700001F0EECF02F0EFCF03F0D9CFE9FFDACFC6
:10308000EAFF0050EE5C0150EE580250EE5803503B
:10309000EE5801E3D5D0100EDBCFE9FF110EDBCFE8
:1030A000EAFF220EE926000EEA22DFCFEEFF010E34
:1030B000DBCFEEFF020EDBCFEEFF030EDBCFEEFF2A
:1030C000100EDBCFE9FF110EDBCFEAFF160EE9266B
:1030D000000EEA22040EDB50EE26050EDB50EE2237
:1030E000060EDB50EE22070EDB50EE22D950FA0F0F
:1030F000E96EFF0EDA20EA6E040EDB50EE5E050E7E
:10310000DB50EE5A060EDB50EE5A070EDB50EE5A3D
:103110005BD7100EDBCFE9FF110EDBCFEAFF160EF7
:10312000E926000EEA22FA0EDB50EE26FB0EDB50FB
:10313000EE22FC0EDB50EE22FD0EDB50EE22D9CF4C
:10314000E9FFDACFEAFFEECFE6FFEECFE6FFEECF04
:10315000E6FFEFCFE6FF66EC03F0E552E552E552FD
:10316000E552080E3DC0DBFF090E3EC0DBFF0A0E34
:103170003FC0DBFF0B0E40C0DBFF080EDBCF00F0D3
:10318000090EDBCF01F00A0EDBCF02F00B0EDBCF16
:1031900003F0005001100210031052E0100EDBCFBC
:1031A000E9FF110EDBCFEAFF160EE926000EEA2238
:1031B000EECF00F0EECF01F0EECF02F0EFCF03F054
:1031C000090ED8900332023201320032E806F9E1EA
:1031D000100EDBCFE9FF110EDBCFEAFF020EE9266E
:1031E000000EEA22EF04056A066A076AE850001634
:1031F000055001160650021607500316D950080F45
:10320000E96E000EDA20EA6EEE500026EE50012242
:10321000EE500222EE500322100EDBCFE9FF110E1A
:10322000DBCFEAFF260EE926000EEA2200C0EEFF01
:1032300001C0EEFF02C0EEFF03C0EEFF000E09D09A
:10324000100EDBCFE9FF110EDBCFEAFFEE52EF6A83
:10325000010E006E120EE15C02E2E16AE552E16EDF
:0E3260000050E552E5CFDAFFE7CFD9FF1200AC
:02326E000F014E
:10327000006B016B086B096B0A6B0B6BA4C400F04D
:10328000016A026A036A000E006C011E0122021E1E
:103290000222031E0322A5C404F0056A066A076A17
:1032A000180ED8900436053606360736E806F9E1DA
:1032B0000450002605500122065002220750032226
:1032C000A6C408F0096A0A6A0B6A100ED89008367C
:1032D00009360A360B36E806F9E10850002609508F
:1032E00001220A5002220B500322A7C43DF03E6A7D
:1032F0003F6A406A426A010E436E446A456A62EC64
:1033000044F0005039240F010C6F01503A200D6F2A
:1033100002503B200E6F03503C200F6F0CCFE6FF96
:103320000DCFE6FF0ECFE6FFE66E0CCFE6FF0DCF2A
:10333000E6FF0ECFE6FFE66ED00E006E820E016E47
:10334000026A00C0E6FFE66E02C0E6FF800EE66E8F
:10335000000EE66E7BEC43F0036E0D0EE15C02E2C4
:10336000E16AE552E16E0350800EE66E000EE66EF5
:10337000C7EC41F0E552E552306A316A326A336A8D
:10338000346A356A020E366E0F01146B809012009B
:10339000D9CFE6FFDACFE6FFE1CFD9FFE2CFDAFF00
:1033A000E652FB0EDB5001E062DFDF6AFC0EDB5011
:1033B00007E0FD0EDB507F0BE76EFD0EE7CFDBFF76
:1033C000FC0EDB506BE0FD0EDB50040804E0FD0E4C
:1033D000DB50140803E1070EDF6EABD0FD0EDB50AF
:1033E0003F0802E1316A23D0FD0EDB505F0810E098
:1033F000400EF36EFD0EDBCFF4FFF350F45C0AE3F6
:10340000FD0EDB505E0806E3FD0EDB50400802E0D7
:10341000306A0DD0FD0EDB50400803E1010E306E26
:1034200006D0FD0EDB50200804E1010E316E336A38
:1034300032D0FD0EDB50650806E1315004E0346AFD
:10344000356A010E27D0FD0EDB506E0802E1020E38
:10345000336EFD0EDB50700806E1305004E0346A34
:10346000356A030E336EFD0EDB50700807E13150F4
:1034700005E08080346A356A040E0CD0FD0EDB5006
:1034800072080CE131500AE080802A0E346E1C0E66
:10349000356E050E336EF36AF46A53D03350050A65
:1034A00041E0010A3CE0070A15E0010A0AE0030ACC
:1034B00002E0010A41D0FD0EDBCFE6FF49D8E5521C
:1034C0002CD08080FD0EDBCFE6FFC0D9E552DF6E49
:1034D000336A32D08080E66A010EE66EE66A000E3C
:1034E000E66E020EE66E38EC42F0006E050EE15C10
:1034F00002E2E16AE552E16E0050020E1E101E6EFD
:1035000036C000F2010EE66EE66AAAEC3DF0E55226
:10351000E552FD0E1E141E6E080EDF6E0DD080905B
:10352000DF6A0AD0FD0EDB50080806E18090DF6AF2
:10353000366A336A346A356ADF50016AF36E01C055
:10354000F4FFE552E552E5CFDAFFE7CFD9FF1200ED
:10355000D9CFE6FFDACFE6FFE1CFD9FFE2CFDAFF3E
:10356000E652DF6A2A0E341802E11C0E351801E11A
:1035700065D10F0E341802E1270E351801E15ED136
:10358000760E341802E10E0E351801E153D1750E96
:10359000341802E10E0E351801E147D1AC0E341893
:1035A00002E10D0E351801E149D1480E341802E14F
:1035B0000D0E351801E136D10C0E341802E1070E5C
:1035C000351801E129D10B0E341802E1070E351828
:1035D00001E11BD10A0E341802E1070E351801E192
:1035E0000FD1090E341802E1070E351801E103D19D
:1035F000EE0E341802E1030E351801E1A8D0ED0EED
:10360000341802E1030E351801E19AD0EC0E34189B
:1036100002E1030E351801E18ED0EB0E341802E101
:10362000030E351801E182D0EA0E341802E1030ED0
:10363000351801E176D0E90E341802E1030E351891
:103640006BE0345001E0FAD0355001E0F7D0FD0EC8
:10365000DB5005E1315003E0DF6A0A0E08D0FD0EB1
:10366000DB50020806E1315004E0DF6A140E346ECC
:10367000D7D0200EF36EFD0EDBCFF4FFF350F45CD9
:103680000DE3FD0EDB502F0809E3315007E0FD0E7E
:10369000DB50E00F0F01006FDF6AC1D0400EF36E08
:1036A000FD0EDBCFF4FFF350F45C0DE3FD0EDB50B9
:1036B0004F0809E3315007E0FD0EDB50C00F0F014A
:1036C000016FDF6AAFD0FD0EDB50350807E13150E6
:1036D00005E0DF6AAC0E346E0D0E0AD0FD0EDB5035
:1036E0000D0808E1315006E0DF6ABC0E346E020EB0
:1036F000356EA3D0FD0EDB50100804E1315002E01E
:10370000E90E22D0FD0EDB50180801E097D03150B1
:1037100001E194D0090E7DD0FD0EDBCF02FFEA0E51
:1037200013D0FD0EDBCF03FFEB0E0ED0FD0EDBCF73
:1037300004FFEC0E09D0FD0EDBCF05FFED0E04D02B
:10374000FD0EDBCF06FFEE0E346E030E71D0FD0EC4
:10375000DBCF07FF04CF00F0016A026A036A000EA4
:10376000006C011E0122021E0222031E032205CF4D
:1037700004F0056A066A076A180ED8900436053602
:1037800006360736E806F9E1045000260550012206
:10379000065002220750032206CF08F0096A0A6A7F
:1037A0000B6A100ED890083609360A360B36E80632
:1037B000F9E108500026095001220A5002220B505C
:1037C000032207CF3DF03E6A3F6A406A426A010E1B
:1037D000436E446A456A62EC44F0005039240F019C
:1037E000086F01503A20096F02503B200A6F0350C6
:1037F0003C200B6F17D0FD0EDBCF13FF0A0E09D054
:10380000FD0EDBCF12FF0B0E04D0FD0EDBCF11FF40
:103810000C0E346E070E0CD0FD0EDBCF10FF346A99
:10382000356A0BD0346A356A09D0760E346E0E0EC6
:10383000356E04D0346A356ADF6A8090DF50E55215
:10384000E552E5CFDAFFE7CFD9FF1200D9CFE6FF87
:10385000DACFE6FFE1CFD9FFE2CFDAFFE6520F0E73
:10386000341802E1270E351823E0BC0E341802E1AB
:10387000020E351819E0AC0E341802E10D0E3518A1
:1038800011E0140E341801E1355007E00A0E341827
:103890000EE135500CE1030E08D0050EDF6E346AE0
:1038A000356A06D0010E01D0020EDF6E01D0DF6A4C
:1038B000DF50E552E552E5CFDAFFE7CFD9FF12003E
:1038C000FD0E1E141E6E050EE66EE66A840EE66E92
:1038D000040EE66E000EE66E020EE66E0DEC42F091
:1038E000006E060EE15C02E2E16AE552E16E005014
:1038F000050EE66EE66AAAEC3DF0E552E552130EBF
:10390000E66EE66A890EE66E040EE66E000EE66E60
:10391000020EE66E0DEC42F0006E060EE15C02E275
:10392000E16AE552E16E0050130EE66EE66AAAEC1B
:103930003DF0E552E552020E1E101E6E0D0EE66EB3
:10394000E66A9C0EE66E040EE66E000EE66E020E51
:10395000E66E0DEC42F0006E060EE15C02E2E16AFA
:10396000E552E16E00500D0EE66EE66AAAEC3DF0FF
:10397000E552E552FD0E1E141E6E80901200020EDE
:103980001E101E6EE66A010EE66EE66A000EE66E18
:10399000020EE66E38EC42F0006E050EE15C02E2CB
:1039A000E16AE552E16E00500201110E006F0169FB
:1039B0000F0114A503D00201010E046F0F0114A121
:1039C00003D00201020E066F0F0114A303D00201FF
:1039D000020E066F82A403D00201080E066F14CFF8
:1039E00036F002CF0BF203CF0CF204CF0DF205CF6D
:1039F0000EF206CF0FF207CF10F2140EE66EE66A53
:103A0000AAEC3DF0E552E552FD0E1E141E6E8090AC
:103A10001200D9CFE6FFDACFE6FFE1CFD9FFE2CF40
:103A2000DAFFE652E652E652E652E65208CFDFFFF0
:103A3000010E09CFDBFF020E0ACFDBFF030E0BCF17
:103A4000DBFF080EE96E0F0EEA6EEE500F010C5D03
:103A5000EE500D59EE500E59EE500F5905E2010E81
:103A6000366E040E1411146F100EE96E0F0EEA6E0E
:103A70000851EE24006E0951EE20016E0A51EE202D
:103A8000026E0B51EE20036E00500C5D01500D597B
:103A900002500E5903500F5905E2010E366E040E06
:103AA0001411146F366AD9CFE9FFDACFEAFFEECFEF
:103AB000E6FFEECFE6FFEECFE6FFEFCFE6FF1DEC31
:103AC00016F0E552E552E552E552E76E040EE7CFF7
:103AD000DBFFDB5006E0010E366E040E0F01141101
:103AE000146F3650016A36C0F3FF01C0F4FF050EB3
:103AF000E15C02E2E16AE552E16EE552E5CFDAFF10
:103B0000E7CFD9FF1200D9CFE6FFDACFE6FFE1CF4A
:103B1000D9FFE2CFDAFF0F0EE12402E3E168E652BB
:103B2000E16E808076DF020EF3CFDBFF030EF4CF71
:103B3000DBFFD950020FE96E000EDA20EA6EEE507C
:103B4000ED1001E0E9D010CF3DF011CF3EF012CFE3
:103B50003FF013CF40F0426A010E436E446A456A5B
:103B6000C7EC44F00B0E3DC0DBFF0C0E3EC0DBFF8C
:103B700010CF3DF011CF3EF012CF3FF013CF40F009
:103B8000426A010E436E446A456AC7EC44F00D0E6A
:103B900039C0DBFF0E0E3AC0DBFFFD0E1E141E6E99
:103BA000040EDB6A050EDB6A060EDB6A070EDB6AB3
:103BB000DE6ADD6ADECF00F0DDCF01F00B0EDBCF79
:103BC00002F00C0EDBCF03F001500318E8AE02D078
:103BD000033404D00250005C0350015870E20B0E15
:103BE000DBCF00F00C0EDBCF01F00006000E015A17
:103BF0000050DF1810E10150DE52DD180CE1D95001
:103C00000D0FE96E000EDA20EA6EEE50ED1003E1C2
:103C1000020E1E101E6ED950090FE66E000EDA203D
:103C2000E66EE66A010EE66E000EE66E020EE66EC7
:103C300035EC10F0006E060EE15C02E2E16AE5523E
:103C4000E16E0050E76E080EE7CFDBFFDB5064E16A
:103C5000090EDBCFE6FF0A0EDBCFE6FFAAEC3DF054
:103C6000E552E552090EDBCF00F00A0EDBCF01F082
:103C7000026A036AD950040FE96E000EDA20EA6E78
:103C8000EE500026EE500122EE500222EE500322AA
:103C9000040E00C0DBFF050E01C0DBFF060E02C0F4
:103CA000DBFF070E03C0DBFF0F01092B000E0A2309
:103CB0000B23DF2A010E01E27DD7DB2A7BD70D0E15
:103CC000DBCF00F00E0EDBCF01F0013466E20050D6
:103CD0000008000E015461E2D950090FE66E000E93
:103CE000DA20E66E0D0EDBCFE6FF0E0EDBCFE6FF31
:103CF000000EE66E020EE66E35EC10F0006E060E5B
:103D0000E15C02E2E16AE552E16E0050E76E080E06
:103D1000E7CFDBFFDB500DE0040E0F011411146F31
:103D200098EC22F0020EDBCF00F0030EDBCF01F0A7
:103D30003CD0020E1E101E6E0D0EDBCFE6FF0E0EE7
:103D4000DBCFE6FFAAEC3DF0E552E552090EDBCFF2
:103D500000F00A0EDBCF01F0026A036AD950040FAB
:103D6000E96E000EDA20EA6EEE500026EE500122D7
:103D7000EE500222EE500322040E00C0DBFF050EBF
:103D800001C0DBFF060E02C0DBFF070E03C0DBFF36
:103D90000F01092B000E0A230B23FD0E1E141E6EAD
:103DA000366A80903650006E016A00C0F3FF01C091
:103DB000F4FF0F0EE15C02E2E16AE552E16EE552CA
:103DC000E5CFDAFFE7CFD9FF1200D9CFE6FFDACF90
:103DD000E6FFE1CFD9FFE2CFDAFF0F0EE12402E3E5
:103DE000E168E652E16E366A14DE0B0EF3CFDBFFBC
:103DF0000C0EF4CFDBFFD9500B0FE96E000EDA206A
:103E0000EA6EEE50ED1007E00B0EDBCF00F00C0E6B
:103E1000DBCF01F0A4D0060EDB6A070EDB6A080ECA
:103E2000DB6A090EDB6A010EDE6EDD6AD9CFE9FFBF
:103E3000DACFEAFFEE50ED1001E196D00001AD6B54
:103E4000AE6B7FEC3EF00B0EF3CFDBFF0C0EF4CF2E
:103E5000DBFFADC000F0AEC001F0026A036AD950CA
:103E6000060FE96E000EDA20EA6EEE500026EE50E4
:103E70000122EE500222EE500322060E00C0DBFFAC
:103E8000070E01C0DBFF080E02C0DBFF090E03C0F6
:103E9000DBFFD950060FE96E000EDA20EA6E0F0143
:103EA0001051EE5C1151EE581251EE581351EE586C
:103EB00002E3DE6ADD6AD9500B0FE96E000EDA20EC
:103EC000EA6EFE0EEE1804E1ED5002E1DE6ADD6AF4
:103ED00081BC02D0DE6ADD6A0001000EAD5D010E1C
:103EE000AE592DE2ADC000F0AEC001F0000ED8809A
:103EF0000056010E015600C0E6FF01C0E6FFADC04E
:103F0000E9FFAEC0EAFFE906000EEA5A000EE92614
:103F1000010EEA22EF50E66E000EAD25026E010E94
:103F2000AE21036E02C0E6FFE66E38EC42F0046E8E
:103F3000050EE15C02E2E16AE552E16E045096D8BA
:103F40000A0EF3CFDBFFDB5001E170D7010E366EB6
:103F5000040E0F011411146F3650006E016A00C078
:103F6000F3FF01C0F4FF07D082A402D0010E366E29
:103F70008090F36AF46A0F0EE15C02E2E16AE552B6
:103F8000E16EE552E5CFDAFFE7CFD9FF1200E66A2E
:103F9000010EE66EE66A000EE66E020EE66E38EC84
:103FA00042F0006E050EE15C02E2E16AE552E16E6C
:103FB000005036C000F2010EE66EE66AAAEC3DF053
:103FC000E552E552366A12000F01086B096B0A6B65
:103FD0000B6B146B106B116B126B136B8090366A4A
:103FE0001200D9CFE6FFDACFE6FFE1CFD9FFE2CF6B
:103FF000DAFFE652E652E652E652E6520F01092B8C
:10400000000E0A230B2308CFDFFF010E09CFDBFFD1
:10401000020E0ACFDBFF030E0BCFDBFFD9CFE9FF88
:10402000DACFEAFFEECFE6FFEECFE6FFEECFE6FF18
:10403000EFCFE6FF1DEC16F0E552E552E552E552F2
:10404000E76E040EE7CFDBFFDB5003E0010E366EB8
:1040500001D0366A050EE15C02E2E16AE552E16EEA
:10406000E552E5CFDAFFE7CFD9FF1200D9CFE6FF5F
:10407000DACFE6FFE1CFD9FFE2CFDAFF130EE1247A
:1040800002E3E168E652E16E08CF3DF009CF3EF071
:104090000ACF3FF00BCF40F0426A010E436E446AF4
:1040A000456AC7EC44F00A0E3DC0DBFF0B0E3EC074
:1040B000DBFF0C0E3FC0DBFF0D0E40C0DBFF110E1F
:1040C000DB6A120EDB6AA5DC040EF3CFDBFF050E04
:1040D000F4CFDBFFD950040FE96E000EDA20EA6E50
:1040E000EE50ED1005E0040EDBCF00F0050E0ED211
:1040F0000A0EDBCF00F00B0E0C0E0D0E010E00169B
:10410000016A026A036A005001100210031001E004
:10411000ACD00A0EDBCF00F00B0EDBCF01F00C0EA3
:10412000DBCF02F00D0EDBCF03F0D890033202326A
:1041300001320032090ED8900036013602360336BD
:10414000E806F9E1012A000E02220322060E00C051
:10415000DBFF070E01C0DBFF080E02C0DBFF090E0C
:1041600003C0DBFFD950060FE96E000EDA20EA6EBD
:10417000EECFE6FFEECFE6FFEECFE6FFEFCFE6FFB6
:104180001DEC16F0E552E552E552E552E76E100ED1
:10419000E7CFDBFFDB5007E0100EDBCF00F0016A5A
:1041A00000AEB6D1A3D1D9500E0FE66E000EDA20C4
:1041B000E66EE66A010EE66E000EE66E030EE66E31
:1041C00035EC10F0006E060EE15C02E2E16AE552A9
:1041D000E16E0050E76E100EE7CFDBFFDB5007E02B
:1041E000100EDBCF00F0016A00AE92D17FD1060E37
:1041F000DBCF00F0070EDBCF01F0080EDBCF02F0C3
:10420000090EDBCF03F00106000E025A035A060E18
:1042100000C0DBFF070E01C0DBFF080E02C0DBFFA2
:10422000090E03C0DBFFD950060FE96E000EDA203D
:10423000EA6EEECFE6FFEECFE6FFEECFE6FFEFCF82
:10424000E6FF1DEC16F0E552E552E552E552E76E49
:10425000100EE7CFDBFFDB5001E1B8D0100EDBCF53
:1042600000F0016A00AE54D141D10A0EDBCF3DF01F
:104270000B0EDBCF3EF00C0EDBCF3FF00D0EDBCF95
:1042800040F0D89040323F323E323D32426A020E18
:10429000436E446A456A62EC44F0060E39C0DBFFA7
:1042A000070E3AC0DBFF080E3BC0DBFF090E3CC027
:1042B000DBFFD950060FE96E000EDA20EA6EEECF72
:1042C000E6FFEECFE6FFEECFE6FFEFCFE6FF1DEC19
:1042D00016F0E552E552E552E552E76E100EE7CFD3
:1042E000DBFFDB5007E0100EDBCF00F0016A00AE11
:1042F0000FD1FCD0D9500E0FE66E000EDA20E66E1C
:10430000E66A010EE66E000EE66E030EE66E35EC12
:1043100010F0006E060EE15C02E2E16AE552E16E29
:104320000050E76E100EE7CFDBFFDB5007E0100E0A
:10433000DBCF00F0016A00AEEBD0D8D0D950060F29
:10434000E96E000EDA20EA6EEECFE6FFEECFE6FF72
:10435000EECFE6FFEFCFE6FF1DEC16F0E552E5529B
:10436000E552E552E76E100EE7CFDBFFDB5007E0CA
:10437000100EDBCF00F0016A00AECAD0B7D082B415
:104380001BD0D9500E0FE66E000EDA20E66EE66AFC
:10439000010EE66E000EE66E030EE66EFDEC12F008
:1043A000006E060EE15C02E2E16AE552E16E005049
:1043B000E76E100EE7CFDBFF100EDB5007E0100EAC
:1043C000DBCF00F0016A00AEA3D090D082B41BD046
:1043D000D9500E0FE66E000EDA20E66EE66A010E88
:1043E000E66E000EE66E010EE66EFDEC12F0006E5B
:1043F000060EE15C02E2E16AE552E16E0050E76E12
:10440000100EE7CFDBFF100EDB500EE0010EF36E57
:10441000110EF3CFDBFF120EDB6A100EDBCF00F0C4
:10442000016A00AE75D062D00A0EDBCF00F00B0E31
:104430000C0E0D0E010E0016016A026A036A00508E
:1044400001100210031027E182B41BD0D9500E0FC7
:10445000E66E000EDA20E66EE66A010EE66E000EEB
:10446000E66E030EE66EFDEC12F0006E060EE15CE9
:1044700002E2E16AE552E16E0050E76E100EE7CF0E
:10448000DBFF100EDB5007E0100EDBCF00F0016AFF
:1044900000AE3ED02BD082B419D0D9500E0FE66EAC
:1044A000000EDA20E66E000EE66EE66AE66EE66A5A
:1044B000FDEC12F0006E060EE15C02E2E16AE552EC
:1044C000E16E0050E76E100EE7CFDBFF100EDB5001
:1044D0000FE0010EF36E110EF3CFDBFF120EDB6A5D
:1044E000100EDBCF00F0016A00AE12D0016810D0D0
:1044F000D950110FE96E000EDA20EA6EEE50ED1081
:1045000001E16FDD110EDBCF00F0120EDBCF01F009
:1045100000C0F3FF01C0F4FF130EE15C02E2E16AA8
:10452000E552E16EE552E5CFDAFFE7CFD9FF1200A1
:10453000E66A010EE66EE66A000EE66E020EE66EB2
:1045400038EC42F0006E050EE15C02E2E16AE552F1
:10455000E16E00500201010E006F020E1E101E6E71
:10456000010EE66EE66AAAEC3DF0E552E552FD0E5C
:104570001E141E6E1200D9CFE6FFDACFE6FFE1CFA0
:10458000D9FFE2CFDAFFE652E652E6520F01020E01
:10459000116F076F04CF00F0016A026A036A000E10
:1045A000006C011E0122021E0222031E032205CFFF
:1045B00004F0056A066A076A180ED89004360536B4
:1045C00006360736E806F9E10450002605500122B8
:1045D000065002220750032206CF08F0096A0A6A31
:1045E0000B6A100ED890083609360A360B36E806E4
:1045F000F9E108500026095001220A5002220B500E
:10460000032207CF3DF03E6A3F6A406A426A010ECC
:10461000436E446A456A62EC44F0005039240F014D
:10462000086F01503A20096F02503B200A6F035077
:104630003C200B6FDE6ADD6ADECF00F0DDCF01F0DB
:10464000140E005C000E015851E2E66ADECFE9FF6D
:10465000DDCFEAFF010EE926000EEA22AD0EE926C3
:10466000040EEA22EF50E66EDECFE9FFDDCFEAFF6F
:10467000AD0EE926040EEA22EF50E66EC8EC19F002
:10468000E552E552E552020EF3CFDBFFDBCFE6FF4A
:10469000E66AC80E006E820E016E026A00C0E6FF76
:1046A000E66E02C0E6FF800EE66E000EE66E7BEC64
:1046B00043F0036E070EE15C02E2E16AE552E16E4F
:1046C0000350800EE66E000EE66EC7EC41F0E55238
:1046D000E552DECF00F0DDCF01F0020E0026000E25
:1046E000012200C0DEFF01C0DDFFA6D7E552E55282
:0E46F000E552E552E5CFDAFFE7CFD9FF120021
:0246FE00D9CF12
:10470000E6FFDACFE6FFE1CFD9FFE2CFDAFF0A0E0C
:10471000E12402E3E168E652E16EDF6A010EDB6A42
:10472000020EDB6A030EDB6A090EDB6A070E966E69
:104730000F01010E1F6F0F01206B929292948082E5
:10474000810ED56EC70ED56EF29474EC41F0650EF5
:10475000006E820E016E026A00C0E6FFE66E02C0C5
:10476000E6FF800EE66E000EE66E7BEC43F0036E15
:10477000050EE15C02E2E16AE552E16E0350800E53
:10478000E66E000EE66EC7EC41F0E552E552480ECB
:10479000E66E820EE66E510EE66E820EE66E5D0EDF
:1047A000006E820E016E026A00C0E6FFE66E02C075
:1047B000E6FF800EE66E000EE66E7BEC43F0036EC5
:1047C000090EE15C02E2E16AE552E16E0350800EFF
:1047D000E66E000EE66EC7EC41F0E552E552010EC2
:1047E000E66EE66A370E006E820E016E026A00C047
:1047F000E6FFE66E02C0E6FF800EE66E000EE66E95
:104800007BEC43F0036E070EE15C02E2E16AE552E5
:10481000E16E0350800EE66E000EE66EC7EC41F0CE
:10482000E552E552FC50E66EE66A2A0E006E820EF4
:10483000016E026A00C0E6FFE66E02C0E6FF800E6F
:10484000E66E000EE66E7BEC43F0036E070EE15C55
:1048500002E2E16AE552E16E0350800EE66E000E60
:10486000E66EC7EC41F0E552E5528450E66EE66A2A
:104870001E0E006E820E016E026A00C0E6FFE66E3A
:1048800002C0E6FF800EE66E000EE66E7BEC43F0A3
:10489000036E070EE15C02E2E16AE552E16E03504D
:1048A000800EE66E000EE66EC7EC41F0E552E55272
:1048B000070E8414E76E090EE7CFDBFF0001A86B3B
:1048C000A96BAA6BAB6B6DEC43F00E0E006E820E03
:1048D000016E026A00C0E6FFE66E02C0E6FF800ECF
:1048E000E66E000EE66E7BEC43F0036E050EE15CB7
:1048F00002E2E16AE552E16E0350800EE66E000EC0
:10490000E66EC7EC41F0E552E552F40EE66E010E9C
:10491000E66E10EC43F0E552E552808406EC29F097
:10492000F3CFDBF0F3CF00F0016A00BE016800C0F6
:10493000E6FF01C0E6FFF60E026E810E036E046A0A
:1049400002C0E6FFE66E04C0E6FF800EE66E000ED3
:10495000E66E7BEC43F0056E070EE15C02E2E16A75
:10496000E552E16E0550800EE66E000EE66EC7EC75
:1049700041F0E552E5520001DB510EE0DBC000F0F2
:10498000016A00BE016800C0E6FF01C0E6FF1EEC40
:104990002CF0E552E552FFD793EC29F00001FB51D2
:1049A0001CE0090EDBCFE6FFE66AE70E006E810E23
:1049B000016E026A00C0E6FFE66E02C0E6FFE10E8D
:1049C000E66E000EE66E7BEC43F0036E070EE15CD4
:1049D00002E2E16AE552E16E03500F011F511EE051
:1049E000D70E006E810E016E026A00C0E6FFE66E11
:1049F00002C0E6FF800EE66E000EE66E7BEC43F032
:104A0000036E050EE15C02E2E16AE552E16E0350DD
:104A10000001020EAF6F0001210E1DD0C70E006E07
:104A2000810E016E026A00C0E6FFE66E02C0E6FF7C
:104A3000800EE66E000EE66E7BEC43F0036E050E14
:104A4000E15C02E2E16AE552E16E03500001010E11
:104A5000AF6F0001040EB06F800EE66E000EE66EC2
:104A6000C7EC41F0E552E552080EDB6A73EC3DF00D
:104A7000E10EE66E000EE66E1DEC0FF0E552E5521B
:104A80000001DC6FE850DB6FDC51E66EE66AE10E98
:104A9000E66E000EE66EB20E006E810E016E026AC8
:104AA00000C0E6FFE66E02C0E6FF800EE66E000E76
:104AB000E66E7BEC43F0036E090EE15C02E2E16A14
:104AC000E552E16E0350800EE66E000EE66EC7EC16
:104AD00041F0E552E5520001DB513CE0DBC000F063
:104AE000016A00BE016800C0E6FF01C0E6FF1EECDF
:104AF0002CF0E552E5520001FB0528E1070E841475
:104B0000006E090EDB50005C21E0070E8414E76E96
:104B1000090EE7CFDBFFDBCFE6FFE66AE70E006EAC
:104B2000810E016E026A00C0E6FFE66E02C0E6FF7B
:104B3000E10EE66E000EE66E7BEC43F0036E070EB0
:104B4000E15C02E2E16AE552E16E03505FDBF3CF24
:104B5000DBF08ED782A420D0980E006E810E016EFD
:104B6000026A00C0E6FFE66E02C0E6FF800EE66E57
:104B7000000EE66E7BEC43F0036E050EE15C02E294
:104B8000E16AE552E16E0350800EE66E000EE66EBD
:104B9000C7EC41F0E552E552B6EC2CF037EC19F0D9
:104BA000060EDB6A070EDB6A8250020B01E0D6D0EC
:104BB000D950060FE96E000EDA20EA6E050EEE18E7
:104BC00001E1ED5001E1CAD00001FB0529E1070E2A
:104BD0008414006E090EDB50005C22E0070E841482
:104BE000E76E090EE7CFDBFFDBCFE6FFE66AE70EF5
:104BF000006E810E016E026A00C0E6FFE66E02C022
:104C0000E6FFE10EE66E000EE66E7BEC43F0036E0F
:104C1000070EE15C02E2E16AE552E16E03509ED0CC
:104C20000001AD6BAE6B80747FEC3EF0080EF3CFED
:104C3000DBFFDB5009E0080EDB50006E016AFF0E5F
:104C4000001808E1015006E10001000ED880AD55C2
:104C5000000EAE550001DB6B0F011F512AE0080E5C
:104C6000DB50070802E1E4EC1FF0080EDB0402E170
:104C700060EC1CF0080EDB50020802E1BFEC1CF0F7
:104C8000080EDB50030808E183EC1DF0060EF3CF9D
:104C9000DBFF070EF4CFDBFF080EDB50050832E127
:104CA000E5EC1EF0060EF3CFDBFF070EF4CFDBFFC3
:104CB00029D0080EDB50070802E151EC32F0080E53
:104CC000DB50020802E113EC2EF0080EDB0402E1D7
:104CD00030EC2EF0080EDB50030802E1FBEC2EF066
:104CE000080EDB50040802E11BEC32F0080EDB502A
:104CF000050802E16AEC2FF0080EDB50060802E11D
:104D000039EC32F00001A85101E14ED7A851E66E0E
:104D1000E66AA80EE66E000EE66E890E006E810E43
:104D2000016E026A00C0E6FFE66E02C0E6FF800E7A
:104D3000E66E000EE66E7BEC43F0036E090EE15C5E
:104D400002E2E16AE552E16E0350800EE66E000E6B
:104D5000E66EC7EC41F0E552E55226D781BC1BD088
:104D6000750E006E810E016E026A00C0E6FFE66EEF
:104D700002C0E6FF800EE66E000EE66E7BEC43F0AE
:104D8000036E050EE15C02E2E16AE552E16E03505A
:104D900081BC19D0FDD7630E006E810E016E026AD0
:104DA00000C0E6FFE66E02C0E6FF800EE66E000E73
:104DB000E66E7BEC43F0036E050EE15C02E2E16A15
:104DC000E552E16E0350800EE66E000EE66EC7EC13
:104DD00041F0E552E5528092E80EE66E030EE66E73
:104DE00010EC43F0E552E5528082E80EE66E030EC9
:104DF000E66E10EC43F0E552E5523AD6D9CFE6FF25
:104E0000DACFE6FFE1CFD9FFE2CFDAFFE652E65292
:104E1000E652E652E652FA0EDBCFE6FFFB0EDBCFA0
:104E2000E6FFFC0EDBCFE6FFFD0EDBCFE6FF540E08
:104E3000006E810E016E026A00C0E6FFE66E02C0DF
:104E4000E6FF800EE66E000EE66E7BEC43F0036E2E
:104E5000090EE15C02E2E16AE552E16E0350800E68
:104E6000E66E000EE66EC7EC41F0E552E552020E2A
:104E7000DB6A030EDB6A020EDBCF00F0030EDBCF32
:104E800001F0D890015004E6500E005C000E01586D
:104E900001E390D1020EDBCF02F0030EDBCF03F073
:104EA000040ED89002360336E806FBE1FA0EDBCF9B
:104EB00004F0FB0EDBCF05F003500518E8AE02D07E
:104EC000053404D00450025C0550035801E372D14C
:104ED000510E006E810E016E026A00C0E6FFE66EA2
:104EE00002C0E6FF800EE66E000EE66E7BEC43F03D
:104EF000036E050EE15C02E2E16AE552E16E0350E9
:104F0000800EE66E000EE66EC7EC41F0E552E5520B
:104F1000DE6ADD6ADECF00F0DDCF01F0D89001500F
:104F200004E6100E005C000E01586BE2020EDBCFAF
:104F300004F0030EDBCF05F0040ED89004360536DE
:104F4000E806FBE1DE500424026EDD500520036E0E
:104F5000FA0EDBCF06F0FB0EDBCF07F0075003188D
:104F6000E8AE02D0033404D00250065C0350075868
:104F700048E3FC0EDBCF02F0FD0EDBCF03F0DE508A
:104F80000224006EDD500320016E100E3F6E406A59
:104F9000020EDBCF44F0030EDBCF45F09AEC44F079
:104FA00000503D24E96E01503E20EA6E040EEFCF22
:104FB000DBFFDBCFE6FFE66A4B0E006E810E016E73
:104FC000026A00C0E6FFE66E02C0E6FF800EE66EF3
:104FD000000EE66E7BEC43F0036E070EE15C02E22E
:104FE000E16AE552E16E0350800EE66E000EE66E59
:104FF000C7EC41F0E552E552DF2A010E8BE3DB2AD4
:1050000089D7470E006E810E016E026A00C0E6FF6E
:10501000E66E02C0E6FF800EE66E000EE66E7BECEA
:1050200043F0036E050EE15C02E2E16AE552E16ED7
:105030000350800EE66E000EE66EC7EC41F0E552BE
:10504000E552DE6ADD6ADECF00F0DDCF01F0D890F8
:10505000015004E6100E005C000E015801E3A3D0DD
:10506000020EDBCF04F0030EDBCF05F0040ED89068
:1050700004360536E806FBE1DE500424026EDD50FE
:105080000520036EFA0EDBCF06F0FB0EDBCF07F038
:1050900007500318E8AE02D0033404D00250065C77
:1050A0000350075801E27FD0FC0EDBCF02F0FD0E6B
:1050B000DBCF03F0DE500224006EDD500320016ED2
:1050C000100E3F6E406A020EDBCF44F0030EDBCFC2
:1050D00045F09AEC44F000503D24E96E01503E202A
:1050E000EA6EEF50200839E2FC0EDBCF02F0FD0E35
:1050F000DBCF03F0DE500224006EDD500320016E92
:10510000100E3F6E406A020EDBCF44F0030EDBCF81
:1051100045F09AEC44F000503D24E96E01503E20E9
:10512000EA6EEF50E66EE66A440E046E810E056E7E
:10513000066A04C0E6FFE66E06C0E6FF800EE66E75
:10514000000EE66E7BEC43F0076E070EE15C02E2B8
:10515000E16AE552E16E075018D0420E006E810EF2
:10516000016E026A00C0E6FFE66E02C0E6FF800E36
:10517000E66E000EE66E7BEC43F0036E050EE15C1E
:1051800002E2E16AE552E16E0350800EE66E000E27
:10519000E66EC7EC41F0E552E552DF2A010E01E26E
:1051A00052D7DB2A50D7020EDB2A030E01E263D668
:1051B000DB2A61D6510E006E810E016E026A00C0BC
:1051C000E6FFE66E02C0E6FF800EE66E000EE66EBB
:1051D0007BEC43F0036E050EE15C02E2E16AE5520E
:1051E000E16E0350800EE66E000EE66EC7EC41F0F5
:1051F000E552E552050EE15C02E2E16AE552E16E3C
:10520000E552E5CFDAFFE7CFD9FF1200D9CFE6FFAD
:10521000DACFE6FFE1CFD9FFE2CFDAFFE652E6527E
:10522000050EDE6EDD6A0001630EDB6FDECF00F07F
:10523000DDCF01F0013466E200500008000E015499
:1052400061E20001DB515EE0DF06010E01E2DB06F8
:10525000370E006E810E016E026A00C0E6FFE66E38
:1052600002C0E6FF800EE66E000EE66E7BEC43F0B9
:10527000036E050EE15C02E2E16AE552E16E035065
:10528000800EE66E000EE66EC7EC41F0E552E55288
:10529000320EE66EE66A10EC43F0E552E552B10ECE
:1052A000E66E000EE66E11EC0AF0E552E5520001E2
:1052B000DB6F006E016A00BE016800C0E6FF01C03E
:1052C000E6FF240E026E810E036E046A02C0E6FF42
:1052D000E66E04C0E6FF800EE66E000EE66E7BEC26
:1052E00043F0056E070EE15C02E2E16AE552E16E11
:1052F0000550800EE66E000EE66EC7EC41F0E552FA
:10530000E55294D7DBC000F0016A00BE016800C01E
:10531000F3FF01C0F4FFE552E552E552E5CFDAFFB5
:10532000E7CFD9FF1200D9CFE6FFDACFE6FFE1CF12
:10533000D9FFE2CFDAFF200EE12402E3E168E65272
:10534000E16E130E006E810E016E026A00C0E6FF70
:10535000E66E02C0E6FF800EE66E000EE66E7BECA7
:1053600043F0036E050EE15C02E2E16AE552E16E94
:105370000350800EE66E000EE66EC7EC41F0E5527B
:10538000E552EF0EE66E000EE66E1DEC0FF0E552F4
:10539000E5520001DC6FE850DB6FDC51E66EE66A37
:1053A000EF0EE66E000EE66EB20E006E810E016E1E
:1053B000026A00C0E6FFE66E02C0E6FF800EE66EFF
:1053C000000EE66E7BEC43F0036E090EE15C02E238
:1053D000E16AE552E16E0350800EE66E000EE66E65
:1053E000C7EC41F0E552E5520001DB510AE0DBC0B9
:1053F00000F0016A00BE016800C0F3FF01C0F4FFC5
:1054000011D2D9500A0FE66E000EDA20E66EE66A77
:10541000010EE66E000EE66E030EE66E35EC10F041
:10542000006E060EE15C02E2E16AE552E16E0050B8
:105430000001DB6F0A0EDBCFE6FF0B0EDBCFE6FFD2
:10544000030E006E810E016E026A00C0E6FFE66E7A
:1054500002C0E6FF800EE66E000EE66E7BEC43F0C7
:10546000036E070EE15C02E2E16AE552E16E035071
:10547000800EE66E000EE66EC7EC41F0E552E55296
:10548000020EDB6A030EDB6A040EDB6A050EDB6AC2
:10549000060EDB6A070EDB6A060EDBCF00F0070E96
:1054A000DBCF01F0D890015004E60A0E005C000E3C
:1054B000015824E2D9500C0F006E000EDA20016E64
:1054C000060EDB500024E96E070EDB500120EA6E69
:1054D000EF6AD950160F006E000EDA20016E060E2C
:1054E000DB500024E96E070EDB500120EA6EEF6A04
:1054F000060EDB2A070ED0E3DB2ACED7DE6ADD6A92
:10550000DECF00F0DDCF01F00A0EDBCF02F00B0E94
:10551000DBCF03F00250005C0350015801E358D187
:10552000DECFE9FFDDCFEAFF000EE926030EEA2217
:10553000EF500D0801E0E0D0D950160FE66E000ED6
:10554000DA20E66ED9500C0FE66E000EDA20E66E19
:10555000F70E006E800E016E026A00C0E6FFE66E76
:1055600002C0E6FF800EE66E000EE66E7BEC43F0B6
:10557000036E090EE15C02E2E16AE552E16E03505E
:10558000800EE66E000EE66EC7EC41F0E552E55285
:10559000D9500C0FE66E000EDA20E66EF10E006EAA
:1055A000800E016E026A00C0E6FFE66E02C0E6FFF2
:1055B00052EC42F0036E050EE15C02E2E16AE55254
:1055C000E16E035000090DE1D950160FE66E000E92
:1055D000DA20E66E9BEC42F0E552E552F3500F0103
:1055E0001F6FD9500C0FE66E000EDA20E66EEB0E40
:1055F000006E800E016E026A00C0E6FFE66E02C019
:10560000E6FF52EC42F0036E050EE15C02E2E16A55
:10561000E552E16E035000090DE1D950160FE66E18
:10562000000EDA20E66E9BEC42F0E552E552F350B4
:105630000F01206FD9500C0FE66E000EDA20E66ED7
:10564000E40E006E800E016E026A00C0E6FFE66E98
:1056500002C0E6FF52EC42F0036E050EE15C02E28E
:10566000E16AE552E16E035000090DE1D950160FD1
:10567000E66E000EDA20E66E9BEC42F0E552E55253
:10568000F3500001FB6F060EDB6A070EDB6A060EA5
:10569000DBCF00F0070EDBCF01F0D890015004E61D
:1056A0000A0E005C000E015824E2D9500C0F006E67
:1056B000000EDA20016E060EDB500024E96E070EA4
:1056C000DB500120EA6EEF6AD950160F006E000E13
:1056D000DA20016E060EDB500024E96E070EDB5067
:1056E0000120EA6EEF6A060EDB2A070ED0E3DB2A02
:1056F000CED7040EDB6A1BD0DECFE9FFDDCFEAFF99
:10570000000EE926030EEA22EF500A085BE0DECF26
:10571000E9FFDDCFEAFF000EE926030EEA22EF5093
:1057200020080CE1010EF36E040EF3CFDBFF050E33
:10573000DB6A020EDB6A030EDB6A44D0D950040F29
:10574000E96E000EDA20EA6EEE50ED100DE0DECFCD
:10575000E9FFDDCFEAFF000EE926030EEA22EF5053
:10576000E66ED950160F0CD0DECFE9FFDDCFEAFF91
:10577000000EE926030EEA22EF50E66ED9500C0F18
:10578000006E000EDA20016E020EDB500024E96E7E
:10579000030EDB500120EA6EE552E750EF6E020E79
:1057A000DBCF00F0030EDBCF01F0D890015004E610
:1057B0000A0E005C000E015805E2020EDB2A030E01
:1057C00001E3DB2ADF2A010E01E29AD6DB2A98D612
:1057D0000F012051E66EE66A0F011F51E66EE66A80
:1057E000D80E006E800E016E026A00C0E6FFE66E03
:1057F00002C0E6FF800EE66E000EE66E7BEC43F024
:10580000036E090EE15C02E2E16AE552E16E0350CB
:10581000800EE66E000EE66EC7EC41F0E552E552F2
:10582000F36AF46A200EE15C02E2E16AE552E16E9D
:10583000E552E5CFDAFFE7CFD9FF1200D9CFE6FF77
:10584000DACFE6FFE1CFD9FFE2CFDAFF8092E80EB0
:10585000E66E030EE66E10EC43F0E552E5528082F0
:10586000E80EE66E030EE66E10EC43F0E552E552EC
:10587000FC0EDBCF00F0DB06FD0EDBCF01F001E21A
:10588000DB06005001100EE080922C0EE66E010E39
:10589000E66E10EC43F0E552E55280822C0EE66E87
:1058A000010EE1D78092F40EE66E010EE66E10EC6A
:1058B00043F0E552E5528082E552E5CFDAFFE7CFCB
:1058C000D9FF1200D9CFE6FFDACFE6FFE1CFD9FF4B
:1058D000E2CFDAFFE652E652D650026E036AD750A4
:1058E000046E056A3F6A010E406E04C044F005C0B4
:1058F00045F09AEC44F002503D24006E03503E20E7
:1059000000C0DEFFDD6EF250040B01E0010EE66E1A
:10591000E66ADECFE6FFDDCFE6FFC80E006E800E42
:10592000016E026A00C0E6FFE66E02C0E6FF800E6E
:10593000E66E000EE66E7BEC43F0036E090EE15C52
:1059400002E2E16AE552E16E0350800EE66E000E5F
:10595000E66EC7EC41F0E552E552F294E552E552AD
:0C596000E552E5CFDAFFE7CFD9FF1200D7
:04596C00306A316A02
:105970000401FB6BFC6B020EFD6F80901200D9CF0F
:10598000E6FFDACFE6FFE1CFD9FFE2CFDAFFE6525A
:10599000FB0EDB5001E0EADFDF6AFD0EDB507F0B20
:1059A000E76EFD0EE7CFDBFFFC0EDB503BE0FD0EAC
:1059B000DB50040804E0FD0EDB50140804E1070E80
:1059C000DF6E0401F0D0FD0EDB503F0802E1316ACA
:1059D00023D0FD0EDB505F0810E0400EF36EFD0E8D
:1059E000DBCFF4FFF350F45C0AE3FD0EDB50540808
:1059F00006E3FD0EDB50400802E0306A0DD0FD0EDC
:105A0000DB50400803E1010E306E06D0FD0EDB5086
:105A1000200808E1010E316E0401FB6BFC6BF36A98
:105A2000F46AFAD0620E0401FB1902E11B0EFC19A4
:105A300001E1EDD00F0EFB1902E1270EFC1901E187
:105A4000E6D0580EFB1902E11B0EFC1901E1D7D07C
:105A5000F70EFB1902E11A0EFC1901E1D4D0F60E83
:105A6000FB1902E11A0EFC1901E1C5D0F50EFB1974
:105A700002E11A0EFC1901E1BCD0A40EFB1902E1EF
:105A80001A0EFC1901E1B0D09E0EFB1902E11A0EAC
:105A9000FC1901E1A2D09D0EFB1902E11A0EFC19BE
:105AA00001E196D09C0EFB1902E11A0EFC1901E1EE
:105AB0008AD09B0EFB1902E11A0EFC1901E17ED07F
:105AC000920EFB1902E11A0EFC1901E175D0F40ED9
:105AD000FB1902E11A0EFC1969E0C20EFB1902E182
:105AE0001A0EFC195EE0900EFB1902E11A0EFC1969
:105AF0003EE0FB5101E08BD0FC5101E088D0FD0E6F
:105B0000DB50600804E1305002E0030E4BD0FD0E84
:105B1000DB50600804E1315002E0050E43D0FD0E79
:105B2000DB50680806E1315004E0900EFB6F1A0E5E
:105B3000FC6FFD0EDB50680804E1305002E0020EFD
:105B400031D0FD0EDB506A0806E1315004E0F40E5E
:105B5000FB6F1A0EFC6FFD0EDB50700858E13050E1
:105B600056E0040EDF6EFB6BFC6B808050D0FD0EA8
:105B7000DB50020804E1920EFB6F1A0EFC6FFD0E63
:105B8000DB50030804E0FD0EDB50FF0804E18080D9
:105B9000DF6A809008D0FD0EDB50160838E1A40EB5
:105BA0002BD0020EDF6EFB6BFC6B31D0FD0EDB5099
:105BB00005082DE1F50E20D09B0E1ED0FD0EDBCF8B
:105BC000F7F49C0E19D0FD0EDBCFF8F49D0E14D027
:105BD000FD0EDBCFF9F49E0E0FD0FD0EDBCFFAF4F5
:105BE000FB6BFC6B010E03D0FB6BFC6B060EDF6ED8
:105BF0000ED0F70E01D0F70EFB6F1A0E07D0FB6B1D
:105C0000FC6B040EDF6E0F0EFB6F270EFC6FDF5078
:105C1000016AF36E01C0F4FFE552E552E5CFDAFF09
:105C2000E7CFD9FF1200020E1E101E6E0201006B9C
:105C300082A402D0130E0211016B0D0E026F036BD2
:105C400082A402D0600E036F040EE66EE66AAAEC30
:105C50003DF0E552E552FD0E1E141E6E80901200BE
:105C6000D9CFE6FFDACFE6FFE1CFD9FFE2CFDAFF07
:105C7000E652E652E652E652E652F8C400F0016AF5
:105C8000026A036A00AE03D0016802680368040E6A
:105C9000D8900036013602360336E806F9E102C034
:105CA00003F001C002F000C001F0006AD890003695
:105CB000013602360336F9C404F0056A066A076A3B
:105CC00004AE02D00568066806C007F005C006F0FD
:105CD00004C005F0046A040ED89004360536063672
:105CE0000736E806F9E10450002605500122065067
:105CF000022207500322FAC408F0096A0A6A0B6AF2
:105D000008AE02D009680A680AC00BF009C00AF0A0
:105D100008C009F0086A08500026095001220A50FC
:105D200002220B50032200C0DFFF010E01C0DBFF87
:105D3000020E02C0DBFF030E03C0DBFFD9CFE9FF79
:105D4000DACFEAFFEECFE6FFEECFE6FFEECFE6FFDB
:105D5000EFCFE6FF1DEC16F0E552E552E552E552B5
:105D6000E76E040EE7CFDBFFDB5036E0040EDBCF3F
:105D700000F0016A00BE016800C0E6FF01C0E6FF56
:105D8000D9CFE9FFDACFEAFFEECFE6FFEECFE6FFAD
:105D9000EECFE6FFEFCFE6FFB00E026E820E036E8F
:105DA000046A02C0E6FFE66E04C0E6FF800EE66EFF
:105DB000000EE66E7BEC43F0056E0B0EE15C02E23A
:105DC000E16AE552E16E0550800EE66E000EE66E69
:105DD000C7EC41F0E552E5520401FD6B8090050EE1
:105DE000E15C02E2E16AE552E16EE552E5CFDAFFFD
:105DF000E7CFD9FF1200D9CFE6FFDACFE6FFE1CF38
:105E0000D9FFE2CFDAFF090EE12402E3E168E652AE
:105E1000E16E020EDB6A030EDB6A040EDB6A050E1E
:105E2000DB6AD950070FE66E000EDA20E66EE66AEE
:105E3000010EE66E000EE66E020EE66E35EC10F018
:105E4000006E060EE15C02E2E16AE552E16E00508E
:105E5000E76E060EE7CFDBFFFD0E1E141E6E070E6B
:105E6000DBCFE6FF080EDBCFE6FFAAEC3DF0E55204
:105E7000E552070EDBCF00F0080EDBCF01F0026A1F
:105E8000036AD950020FE96E000EDA20EA6EEE5076
:105E90000026EE500122EE500222EE500322020EA6
:105EA00000C0DBFF030E01C0DBFF040E02C0DBFFFE
:105EB000050E03C0DBFF0401FD6B8090090EE15C61
:105EC00002E2E16AE552E16EE552E5CFDAFFE7CFA3
:105ED000D9FF1200D9CFE6FFDACFE6FFE1CFD9FF35
:105EE000E2CFDAFF150EE12402E3E168E652E16E4B
:105EF000F8C400F0016A026A036A00AE03D00168C8
:105F000002680368040ED890003601360236033664
:105F1000E806F9E1D8900036013602360336F9C4B6
:105F200004F0056A066A076A04AE03D005680668CD
:105F30000768040ED8900436053606360736E8069C
:105F4000F9E10450002605500122065002220750B4
:105F50000322FAC408F0096A0A6A0B6A08AE03D081
:105F600009680A680B6808500026095001220A5087
:105F700002220B5003220E0E00C0DBFF0F0E01C0E9
:105F8000DBFF100E02C0DBFF110E03C0DBFF060EAD
:105F9000DB6A070EDB6A080EDB6A090EDB6A010E9C
:105FA000DE6EDD6A0E0EDBCF00F00F0E100E110E4E
:105FB000010E0016016A026A036A00500110021005
:105FC000031001E08DD00E0EDBCF00F00F0EDBCF03
:105FD00001F0100EDBCF02F0110EDBCF03F0D890F2
:105FE0000332023201320032090ED89000360136F7
:105FF00002360336E806F9E1012A000E02220322E6
:106000000A0E00C0DBFF0B0E01C0DBFF0C0E02C04E
:10601000DBFF0D0E03C0DBFFD9500A0FE96E000E47
:10602000DA20EA6EEECFE6FFEECFE6FFEECFE6FF38
:10603000EFCFE6FF1DEC16F0E552E552E552E552D2
:10604000E76E120EE7CFDBFFD950130FE66E000E9E
:10605000DA20E66EE66A010EE66E000EE66E030ECC
:10606000E66E35EC10F0006E060EE15C02E2E16ACD
:10607000E552E16E0050E76E120EE7CFDBFF0A0E2D
:10608000DBCF00F00B0EDBCF01F00C0EDBCF02F00C
:106090000D0EDBCF03F00106000E025A035A0A0E62
:1060A00000C0DBFF0B0E01C0DBFF0C0E02C0DBFFEC
:1060B0000D0E03C0DBFFD9500A0FE96E000EDA2087
:1060C000EA6EEECFE6FFEECFE6FFEECFE6FFEFCFD4
:1060D000E6FF1DEC16F0E552E552E552E55288D098
:1060E0000E0EDBCF3DF00F0EDBCF3EF0100EDBCF00
:1060F0003FF0110EDBCF40F0D89040323F323E32BD
:106100003D32426A020E436E446A456A62EC44F0D4
:106110000A0E39C0DBFF0B0E3AC0DBFF0C0E3BC092
:10612000DBFF0D0E3CC0DBFFD9500A0FE96E000EFD
:10613000DA20EA6EEECFE6FFEECFE6FFEECFE6FF27
:10614000EFCFE6FF1DEC16F0E552E552E552E552C1
:10615000E76E120EE7CFDBFFD950130FE66E000E8D
:10616000DA20E66EE66A010EE66E000EE66E030EBB
:10617000E66E35EC10F0006E060EE15C02E2E16ABC
:10618000E552E16E0050E76E120EE7CFDBFFD9500B
:106190000A0FE96E000EDA20EA6EEECFE6FFEECFD0
:1061A000E6FFEECFE6FFEFCFE6FF1DEC16F0E5527F
:1061B000E552E552E552E76E120EE7CFDBFF82B4FF
:1061C0001BD0D950130FE66E000EDA20E66EE66A99
:1061D000010EE66E000EE66E030EE66EFDEC12F0AA
:1061E000006E060EE15C02E2E16AE552E16E0050EB
:1061F000E76E120EE7CFDBFFD9CFE9FFDACFEAFF78
:10620000EE50ED1001E192D00001AD6BAE6B7FEC72
:106210003EF0120EF3CFDBFFADC000F0AEC001F0D8
:10622000026A036AD950060FE96E000EDA20EA6EA0
:10623000EE500026EE500122EE500222EE500322D4
:10624000060E00C0DBFF070E01C0DBFF080E02C018
:10625000DBFF090E03C0DBFFD950060FE96E000E0D
:10626000DA20EA6E000EEE5C010EEE58000EEE58DB
:10627000000EEE5802E3DE6ADD6A120EDBCF00F09C
:10628000016A00BE0168FE0E001804E1015002E13F
:10629000DE6ADD6A82B41CD0D950130FE66E000EA0
:1062A000DA20E66EADC0E6FFAEC0E6FF000EE66E99
:1062B000010EE66EFDEC12F0006E060EE15C02E2ED
:1062C000E16AE552E16E0050E76E120EE7CFDBFFA8
:1062D000120EDB5091E0120EDBCF00F0016A00BE1F
:1062E000016800C0E6FF01C0E6FFA00E026E820E4C
:1062F000036E046A02C0E6FFE66E04C0E6FF800E8D
:10630000E66E000EE66E7BEC43F0056E070EE15C78
:1063100002E2E16AE552E16E0550800EE66E000E83
:10632000E66EC7EC41F0E552E55266D70E0EDBCFC4
:1063300000F00F0E100E110E010E0016016A026A17
:10634000036A00500110021003101DE182B436D020
:10635000D950130FE66E000EDA20E66EE66A010EE3
:10636000E66E000EE66E030EE66EFDEC12F0006EB9
:10637000060EE15C02E2E16AE552E16E0050E76E72
:10638000120EE7CFDBFF82B419D0D950130FE66E9F
:10639000000EDA20E66E000EE66EE66AE66EE66A4B
:1063A000FDEC12F0006E060EE15C02E2E16AE552DD
:1063B000E16E0050E76E120EE7CFDBFF120EDB50EE
:1063C0002AE0120EDBCF00F0016A00BE016800C0B7
:1063D000E6FF01C0E6FF8B0E026E820E036E046ABA
:1063E00002C0E6FFE66E04C0E6FF800EE66E000E19
:1063F000E66E7BEC43F0056E070EE15C02E2E16ABB
:10640000E552E16E0550800EE66E000EE66EC7ECBA
:1064100041F0E552E5524DD80401FD6B8090150E18
:10642000E15C02E2E16AE552E16EE552E5CFDAFFB6
:10643000E7CFD9FF1200E66A010EE66EE66A000EAB
:10644000E66E020EE66E38EC42F0006E050EE15C80
:1064500002E2E16AE552E16E0050FDC400F2010E75
:10646000E66EE66AAAEC3DF0E552E5520401FD6BEA
:106470001200E66A010EE66EE66A000EE66E020E95
:10648000E66E38EC42F0006E050EE15C02E2E16A75
:10649000E552E16E00500201006B80900401FD6B3B
:1064A00012000401FA6BF96BF86B80900401FD6B2C
:1064B0001200D9CFE6FFDACFE6FFE1CFD9FFE2CF76
:1064C000DAFFE652E652E652E652E6520401FA2BB1
:1064D0000F0EE76EFA19E8AE02D0FA3503D0E75096
:1064E000D880FA550FE2FA6BF92B010EE76EF91915
:1064F000E8AE02D0F93503D0E750D880F95502E272
:10650000F96BF82BF8C400F0016A026A036A00AE66
:1065100003D0016802680368040ED8900036013683
:1065200002360336E806F9E102C003F001C002F0CA
:1065300000C001F0006AD8900036013602360336FA
:10654000F9C404F0056A066A076A04AE02D0056859
:10655000066806C007F005C006F004C005F0046A2E
:10656000040ED8900436053606360736E806F9E1FB
:106570000450002605500122065002220750032233
:10658000FAC408F0096A0A6A0B6A08AE02D0096800
:106590000A680AC00BF009C00AF008C009F0086ACE
:1065A00008500026095001220A5002220B500322F3
:1065B00000C0DFFF010E01C0DBFF020E02C0DBFFE7
:1065C000030E03C0DBFFD9CFE9FFDACFEAFFEECF3E
:1065D000E6FFEECFE6FFEECFE6FFEFCFE6FF1DECE6
:1065E00016F0E552E552E552E552E76E040EE7CFAC
:1065F000DBFFDB5036E0040EDBCF00F0016A00BEAB
:10660000016800C0E6FF01C0E6FFD9CFE9FFDACF9D
:10661000EAFFEECFE6FFEECFE6FFEECFE6FFEFCFED
:10662000E6FFB00E026E820E036E046A02C0E6FF41
:10663000E66E04C0E6FF800EE66E000EE66E7BECB2
:1066400043F0056E0B0EE15C02E2E16AE552E16E99
:106650000550800EE66E000EE66EC7EC41F0E55286
:10666000E5520401FD6B050EE15C02E2E16AE552D0
:0E667000E16EE552E5CFDAFFE7CFD9FF120069
:02667E007BECB3
:1066800038F0FB0EDBCFF3FFDB06F35000090AE026
:10669000C9EC38F0FA0E34EC39F0F3E1011CF1E109
:1066A000010E01D0000EAAEF38F07BEC38F03B0E63
:1066B000E12402E3E168E652E16E010EDB6A020EBC
:1066C000DB6AF90EDBCFF6FFFA0EDBCFF7FFFB0E2E
:1066D000DBCFF8FF0800F550DF6EDF5002E1CEEFB0
:1066E00037F0250EDF5C02E0C1EF37F0030EDB6A06
:1066F000040EDB6A050EDB6A060EDB6A070EDB6A38
:10670000E3EC37F02D0EDF5C0CE02B0EDF5C09E0D4
:10671000200EDF5C06E0230EDF5C03E0300EDF5C62
:106720001AE1DF50300A14E0130A0FE0030A0AE00E
:106730000B0A05E0060AE4E1030EDB80E1D7030E55
:10674000DB82DED7030EDB84DBD7030EDB86D8D7F4
:10675000030EDB88D5D72A0EDF5C1BE1DFEC37F0B8
:106760002DEC38F010E0030EDB803F684068130E1C
:10677000DBCF44F0140EDBCF45F09AEC44F0040E6E
:106780003DC0DBFF03D0130E16EC38F0E3EC37F01E
:106790000BD0090EDB6A84EC38F003E0F8EC38F03B
:1067A000FAD7090E16EC38F0030EDBB0DB982E0E8C
:1067B000DF5C1BE1E3EC37F02A0EDF5C0BE1DFEC82
:1067C00037F02DEC38F003E1130E68EC38F0E3EC11
:1067D00037F00BD0090EDB6A84EC38F003E0F8ECFC
:1067E00038F0FAD7090E68EC38F0680EDF5C07E184
:1067F000E3EC37F0680EDF5C1DE1030E18D0740E79
:10680000DF5C17E07A0EDF5C14E0480EDF5C06E028
:10681000540EDF5C03E05A0EDF5C02E1020E07D08B
:106820006C0EDF5C03E06A0EDF5C04E1010EBBEC82
:1068300038F0C9DBDF506E0A01E17FD31E0A01E1A7
:1068400092D1200A01E18FD13F0A01E149D11A0A10
:1068500001E146D10D0A01E143D1200A01E140D115
:106860003A0A01E13DD1200A01E13AD1260A01E1CB
:1068700035D10D0A01E132D11A0A01E1D9D0200A3D
:106880004AE0300A1FE0460A0EE0250A01E083D301
:10689000D950F90FE96EFF0EDA20EA6E010EEE5EB6
:1068A000000EEE5AEE5AC9EC38F0250EE66E95DB76
:1068B00003E1011C01E169D3C5EC38F001E26BD3BF
:1068C000DB2A69D3080EDB6A040EDB50010806E2FE
:1068D000040EDB048DEC38F0DB508BDB080EDB5054
:1068E00009E0030EDB50010B05E172DB01E04DD343
:1068F000080EDB6A64DBEFCFDFFF3DEC39F003E12C
:10690000011C01E142D3C5EC38F001E3DB2A60DB76
:1069100001E141D33AD3070EDB5002080FE109EC45
:1069200039F0030ED0EC38F00E0EEECFDBFF0F0E79
:10693000EECFDBFF100EEECFDBFF20D0F70EDBCF6C
:1069400003F0F80EDBCF04F0020E035E000E045AD3
:10695000F70E03C0DBFFF80E04C0DBFF03C0E9FF46
:1069600004C0EAFFC0EC38F0026A0E0E00C0DBFF84
:106970000F0E01C0DBFF100E02C0DBFF0E0EDBCFDF
:10698000E6FF0F0EDBCFE6FF100EDBCFE6FF76EC67
:1069900042F0E552E552E552130E3EC0DBFF140E05
:1069A0003FC0DBFF060EDB5005E0130E04EC39F0B0
:1069B00001E26ADB28EC39F002E2130E37DBEBEC84
:1069C00038F006E0040E04EC39F002E2050E2EDB8E
:1069D000030EDBB005D0FCDA01E0D7D2080EDB6A8B
:1069E000090EDB6A0E0EDBCFF6FF0F0EDBCFF7FFD3
:1069F000100EDBCFF8FF0800F550DF6EDF5014E01B
:106A00002EEC39F011E23DEC39F003E1011C01E11B
:106A1000BCD2BBDB01E3DB2A090EDB2AD9500E0F07
:106A2000E96E000ECBDBE7D7D3DA01E1B4D2ADD209
:106A3000C6DA110EEECFDBFF120EEDCFDBFF110E2B
:106A4000DBCFE6FF120EDBCFE6FF68EC42F0E5524B
:106A5000E552130EF3CFDBFF140EF4CFDBFF060E6F
:106A6000DB5004E0130ED0DB01E20EDB28EC39F042
:106A700002E2130EDBDAAFDB05E0040EC5DB02E257
:106A8000050ED4DA030EDBB005D0A2DA01E07DD228
:106A9000080EDB6A090EDB6A110EDBCFE9FF120E6E
:106AA000DBCFEAFFEFCFDFFFDF5014E0D7DB12E2EE
:106AB000E4DB03E1011C01E168D267DB01E3DB2ACF
:106AC000090EDB2A110EDB2ADBCFE9FF120EE8E309
:106AD000DB2AE6D77DDA01E15ED257D2030EDB8EE8
:106AE000070EDB0410E195DB040E5ADB0A0EEECF35
:106AF000DBFF0B0EEECFDBFF0C0EEECFDBFF0D0E40
:106B0000EECFDBFF6CD0070EDB5003082CE1030E49
:106B1000DBAE0DD0B2DA020E76DAEFCF00F0016A0A
:106B2000026A036A00AE39D00168026835D0F70EF8
:106B3000DBCF01F0F80EDBCF02F0020E015E000E9B
:106B4000025AF70E01C0DBFFF80E02C0DBFF01C0E6
:106B5000E9FF02C0EAFFEFCF00F00A0E00C0DBFF42
:106B60000B0EDB6A38D0070EDB50020809E1030E7A
:106B7000DBAE04D059DB02AE10D00ED055DB0DD009
:106B8000030EDBAE12D079DA020E3DDAF9DA026AD0
:106B9000036A01AE02D002680368E2DA0C0E02C09A
:106BA000DBFF0D0E03C0DBFF1AD0F70EDBCF02F0C8
:106BB000F80EDBCF03F0020E025E000E035AF70E52
:106BC00002C0DBFFF80E03C0DBFF02C0E9FF03C019
:106BD000EAFFD6DAC5DA0C0EDB6A0D0EDB6A060EAA
:106BE000DB5005E1010EF36E050EF3CFDBFF150E52
:106BF000DB6A160EDB6AD950370F006E000EDA2002
:106C0000016E390E00C0DBFF3A0E01C0DBFF380E0B
:106C1000DB6A080EDB6A0A0EAEDADF50780A12E091
:106C2000200A10E0280A0CE0200A0AE03F0A06E0E9
:106C30000D0A02E0200A08E1020E05D0080E03D07A
:106C4000080EDF26100E97DA030EDBBE02D0DB92B1
:106C5000DB94DB50800B24E08ADAD890030EEB50F3
:106C6000000A08E6000EEE5C000EEE58000EEE582C
:106C7000000EEE5815E213DA42684368446845682E
:106C800062EC44F00A0E39C0DBFF0B0E3AC0DBFFAA
:106C90000C0E3BC0DBFF0D0E3CC0DBFF2D0E08D001
:106CA000030EDBA202D02B0E03D0DBA408D0200EF3
:106CB000F36E170EF3CFDBFF150EDB2A02D0170E93
:106CC000DB6A050EDB5003E1B7D901E189D0A00EE4
:106CD000006E8A0E016E000E026E070EDBCF03F00F
:106CE000046A056A066A03C042F004C043F005C0A6
:106CF00044F006C045F0D3D9C7EC44F00050392425
:106D0000F36E01503A20F46E02503B20F86EF4CF3F
:106D1000F7FFF3CFF6FF0800090EF5CFDBFF580EA3
:106D2000DF5C0FE1610EF36E090E7BD90AE3200EE2
:106D3000006E090EDBCFE7FF0050E75E090EE7CFDC
:106D4000DBFF070EDBCF00F0016A026A036A0FDA8D
:106D500000C042F001C043F002C044F003C045F05F
:106D6000EECF3DF0EECF3EF0EECF3FF0EFCF40F074
:106D7000C7EC44F040C0EDFF3FC0EDFF3EC0EDFF6B
:106D80003DC0EFFF390EDBCFE9FFDB063A0EDBCF6C
:106D9000EAFF01E2DB06090EDBCFEFFF150EDB2A6F
:106DA0004BD995E1030EDBA61DD06F0EDF5C06E12B
:106DB000C1D918E3150EDB285BDA14D0780EDF5C3E
:106DC00009E0580EDF5C06E0620EDF5C03E0420E75
:106DD000DF5C08E1020EF36E160EF3CFDBFF02D08C
:106DE000150EDB6A030EDB50100B0EE0040EDBCF3A
:106DF00000F0050EDB50D880005406E2060EDB5092
:106E000003E1040EDB5034DA95D90AE2050EDBCF3C
:106E1000E7FF150EDB50E75E050EE7CFDBFF02D084
:106E2000050EDB6A040EDBCF00F0160E45D9D880C4
:106E3000005414E2160EDBCFE6FF150EDBCFE6FFA3
:106E4000040EDBCFE6FF050EDB50E552E75CE552B2
:106E5000D880E754E552D880E7545FD9030EDB5061
:106E6000010B0BE1080EDB5008E0B2D801E08DD039
:106E7000080EDB50BED8080EDB6A170EDB5007E0A9
:106E800088D9170EF1D903E1011C01E17ED0160E5D
:106E9000DB5016E07ED9300EE66E9FD802E1011C71
:106EA00074E077D9DFCFE6FF20EC44F0E552E552FD
:106EB000E552F4CF01F00001F31C02E1011C65E092
:106EC000050EDBCF00F0160EDB50D880005409E22F
:106ED000050EDBCFE7FF160EDB50E75E050EE7CFB2
:106EE000DBFF300EE66E050ECBD94FE1390EDB2A03
:106EF000DBCFE9FF3A0E01E3DB2ADBCFEAFF090E25
:106F0000EFCFDBFFDB500EE044D9090EADD902E133
:106F1000011C3BE0390EDB2ADBCFE9FF3A0EEDE343
:106F2000DB2AEBD755D831E1160EDBCFE6FF080E92
:106F3000C3D8E552E7245DD82ED0070EDB50030AF4
:106F40001CE0010A14E0030A07E07BD9DBCFEEFF67
:106F5000020EDBCFEDFF1FD0F5D8056A03AE02D0DD
:106F6000046805682CD8BCD805C0EEFF14D0EAD858
:106F700003BE046824D8B4D80ED063D9DBCFEFFFAA
:106F80000AD07BD905E1011C03E1F368F46810D055
:106F9000FCD801E3DB2A79D96AEF33F0010EDBCFAD
:106FA00000F0020EDBCF01F000C0F3FF01C0F4FFE0
:106FB0003B0EE15C02E2E16AE552E16ECBD029D9F9
:106FC000020ED0EF38F061D90800F550DF6E1200E4
:106FD000200EE66E080E40EF39F020EC44F0E5524A
:106FE000E552E552F3CF00F0F4CF01F00001F31CBD
:106FF0001200006E016AD950010F4DD90050EE26E3
:107000000150ED221200045E000E055AF70E04C076
:10701000DBFFF80E05C0DBFF04C0E9FF05C0EAFF97
:107020001200DBCFF4FFF350F45C1200DB50E76E8C
:10703000040EE7CFDBFF12000A0EDBCF00F00B0ED1
:10704000DBCF01F00C0EDBCF02F00D0EDBCF03F037
:1070500000500110021003101200130EEECFDBFFE0
:10706000140EEDCFDBFF130EDBCF00F0140EDBCFE1
:1070700001F00001800E01141200F70EDBCF04F0C6
:10708000F80EDBCF05F01200050EDB50E66ED9508E
:10709000130F01D9E552E750EE6EED6A12000A0EA9
:1070A000DBCF3DF00B0EDBCF3EF00C0EDBCF3FF025
:1070B0000D0EDBCF40F01200DBCFE6FF150EDBCF6D
:1070C000E6FF050EDB50E552E724E552E724120007
:1070D000DB50CED8010EF36E060EF3CFDBFF1200AD
:1070E000EE50EFCFEAFFE96E02C0EEFF03C0EEFF05
:1070F00004C0EEFF1200D9CFE6FFDACFE6FFE1CF02
:10710000D9FFE2CFDAFF1200DFCFE6FFE66A02EC3A
:1071100045F0E552E552F3501200E76E080EE7CF56
:10712000DBFF1200EECF00F0EECF01F0EFCF02F068
:10713000036A1200050EDBCF00F0150EDB50D8807D
:1071400000541200010EDBCF02F0020EDBCF03F081
:10715000046A1200E552E5CFDAFFE7CFD9FF12004B
:107160000A0E00C0DBFF0B0E01C0DBFF1200D9507E
:107170000A0F4BEF39F0F36E070EF3CFDBFF12006F
:10718000EECF00F0EFCF01F01200010EDB2A020E6D
:107190001200FC0EDBCFE6FFFD0EDBCFE6FF120098
:1071A000005E000E015AF70E00C0DBFFF80E01C0B2
:1071B000DBFF00C0E9FF01C0EAFF1200DA20EA6E3F
:1071C000EF2AEECFF6FF000EEF22EECFF7FFEF2211
:1071D000EECFF8FF1200040EDBCFE6FF130EDB50FC
:1071E000E552E75C9ADFDB5004DF060EDB5012004D
:1071F000090EDB500A0DF350DF24D00FE76E090EA5
:10720000E7CFDBFFE3EF37F0DB50F36E050E11EF56
:1072100038F0F70EDBCF00F0F80EDBCF01F01200F4
:10722000DFCFE6FFEDEF37F028DF030EECDE92EF65
:1072300038F03FEC33F0E552E552E552E5520009F3
:107240001200BDDEEE50EFCFEAFFE96E010E120034
:10725000130EDB50F36E040E11EF38F0040EDB500A
:10726000F36E090E11EF38F0DBCFE6FFEDEF37F0EC
:10727000E76E050EE7CFDBFF12008BDF10EF39F072
:10728000DBCFE6FF86DF19EF39F0D950F90FE96E51
:10729000FF0EDEEF38F0E96E000EDA20EA6E120023
:1072A000D9CFE6FFDACFE6FFE1CFD9FFE2CFDAFFB1
:1072B000FD0EDB5003E0C66A010E02D0C66A020E64
:1072C000C66E400EC76EC68AE552E5CFDAFFE7CF3D
:1072D000D9FF1200D9CFE6FFDACFE6FFE1CFD9FF21
:1072E000E2CFDAFFE652E652500EDE6EDD6AD9CF0B
:1072F000E9FFDACFEAFFEE06000EED5AEECF00F01E
:10730000EDCF01F000500110F2E1E552E552E552F7
:10731000E5CFDAFFE7CFD9FF1200D9CFE6FFDACF0A
:10732000E6FFE1CFD9FFE2CFDAFFFD0EDB50C96EF9
:10733000C7B0FED7C7A0FED7FD0EC9CFDBFFE55211
:10734000E5CFDAFFE7CFD9FF1200C968C7B0FED793
:10735000C7A0FED7C9501200D9CFE6FFDACFE6FFAB
:10736000E1CFD9FFE2CFDAFFE652E652FD0EDBAE07
:1073700018D0FD0EDB9EE66AE66AE66AE66A770EDC
:10738000E66EEADF006E050EE15C02E2E16AE552BC
:10739000E16E0050E76E010EE7CFDBFFDB50010826
:1073A00074E38280D2DF8290D0DFFD0EDBCFE6FF78
:1073B000B4DFE552F90EDBCF00F0FA0EDBCF01F0BF
:1073C000FB0EDBCF02F0FC0EDBCF03F0180ED890E3
:1073D0000332023201320032E806F9E10050E66E73
:1073E0009CDFE552F90EDBCF00F0FA0EDBCF01F0A7
:1073F000FB0EDBCF02F0FC0EDBCF03F0100ED890BB
:107400000332023201320032E806F9E10050E66E42
:1074100084DFE552F90EDBCF00F0FA0EDBCF01F08E
:10742000FB0EDBCF02F0FC0EDBCF03F0080ED89092
:107430000332023201320032E806F9E10050E66E12
:107440006CDFE552F90EDBCFE6FF67DFE552010E98
:10745000DF6EFD0EDB50400802E1950EDF6EFD0E83
:10746000DB50480802E1870EDF6EDFCFE6FF55DF15
:10747000E5520A0EDF6E69DFE76E010EE7CFDBFF34
:10748000DB50800B02E0DF06F6E1010EDB50E55237
:10749000E552E552E5CFDAFFE7CFD9FF1200D9CFA9
:1074A000E6FFDACFE6FFE1CFD9FFE2CFDAFF090E40
:1074B000E12402E3E168E652E16EE66AF1DEE552BC
:1074C000720ED36E0001FC5113E08250010B10E1EB
:1074D000E66AE66AE66AE66A000EE66EE66A1BDAC5
:1074E000006E060EE15C02E2E16AE552E16E0050D8
:1074F00082800A0EDF6EDF5003E027DFDF06FBD756
:10750000020EDB6AE66AE66AE66AE66A400EE66E44
:1075100023DF006E050EE15C02E2E16AE552E16EF6
:107520000050010801E008D1AA0EE66E010EE66ED9
:10753000E66AE66A480EE66E0FDF006E050EE15C55
:1075400002E2E16AE552E16E0050010801E08DD0EF
:10755000DF6A040EDF5C14E2F8DEE66ED950030F3A
:10756000006E000EDA20016EDF500F010024E96E7C
:10757000000E0120EA6EE552E750EF6EDF2AE9D7F0
:10758000050EDB0401E0D8D0060EDB50AA0801E0AE
:10759000D3D0100EF36E070EF3CFDBFF270EF36E82
:1075A000080EF3CFDBFFD950070FE96E000EDA208B
:1075B000EA6EEE50ED1019E0E66AE66AE66A400E01
:1075C000E66EE90EE66EC8DE006E050EE15C02E2D4
:1075D000E16AE552E16E0050000907E07BDE070E2C
:1075E000DB06080EE0E2DB06DED7D950070FE96EB6
:1075F000000EDA20EA6EEE50ED1001E19DD0E66A51
:10760000E66AE66AE66A7A0EE66EA6DE006E050EA9
:10761000E15C02E2E16AE552E16E0050000901E03E
:107620008BD0DF6A040EDF5C14E28FDEE66ED95089
:10763000030F006E000EDA20016EDF500F010024F0
:10764000E96E000E0120EA6EE552E750EF6EDF2A88
:10765000E9D7030EDB50400B02E00C0E01D0040E04
:10766000E76E020EE7CFDBFF67D0E66AE66AE66AFE
:10767000E66AE90EE66E70DE006E050EE15C02E27F
:10768000E16AE552E16E0050010805E3020EDB6E8F
:10769000DE52E90E07D0010EF36E020EF3CFDBFFD0
:1076A000DE52410EDD6E100EF36E070EF3CFDBFFE0
:1076B000270EF36E080EF3CFDBFFD950070FE96EEC
:1076C000000EDA20EA6EEE50ED1019E0E66AE66A86
:1076D000E66AE66A010EDBCFE6FF3EDE006E050ECF
:1076E000E15C02E2E16AE552E16E0050000907E068
:1076F000F1DD070EDB06080EE0E2DB06DED7D9502F
:10770000070FE96E000EDA20EA6EEE50ED1012E07F
:10771000E66A020EE66EE66AE66A500EE66E1CDE69
:10772000006E050EE15C02E2E16AE552E16E005096
:10773000000902E0020EDB6A020EDBCFFCF0828061
:1077400004DE010EE66EACDDE552D36A020EDB50BC
:1077500002E0000E01D0010E006E090EE15C02E2B3
:10776000E16AE552E16E0050E552E5CFDAFFE7CF7E
:10777000D9FF1200D9CFE6FFDACFE6FFE1CFD9FF7C
:10778000E2CFDAFFE652E652E652E6520001FCB7DB
:1077900012D0D950F80FE96EFF0EDA20EA6E090E0A
:1077A000E76ED890EF36010EEB36020EEB36030E85
:1077B000EB36E706F6E1010EDF6ED950F80FE96E01
:1077C000FF0EDA20EA6EEECFE6FFEECFE6FFEECF59
:1077D000E6FFEFCFE6FF510EE66EBEDD006E050E52
:1077E000E15C02E2E16AE552E16E0050000901E06D
:1077F00081D0400EF36E020EF3CFDBFF9C0EF36ED2
:10780000030EF3CFDBFFA1DDE76E010EE7CFDBFF59
:10781000DB50FF080CE1020EDB06DBCF00F0030EAD
:1078200001E2DB06DBCF01F000500110ECE1010EBC
:10783000DB50FE085FE1F60EDBCF02F0F70EDBCF88
:1078400003F0020ED88002560356F40EDB50025CA1
:10785000006EF50EDB500358016E020E00C0DBFF18
:10786000030E01C0DBFFD950F60FE96EFF0EDA20E0
:10787000EA6EEE50ED100DE068DDF60EDB06DBCFB4
:1078800000F0F70E01E2DB06DBCF01F00050011043
:10789000F3E1D950FC0FE96EFF0EDA20EA6EEE50EC
:1078A000ED101AE052DDE66EFC0EDBCFE9FFDB2ABD
:1078B000FD0EDBCFEAFF01E3DB2AE552E750EF6E76
:1078C000F40EDB06DBCF00F0F50E01E2DB06DBCFCA
:1078D00001F000500110E6E138DD020EDB06DBCFDF
:1078E00000F0030E01E2DB06DBCF01F000500110D7
:1078F000F3E1DF6A828029DDDF50006E040EE15C77
:1079000002E2E16AE552E16E0050E552E5CFDAFFAE
:10791000E7CFD9FF1200D9CFE6FFDACFE6FFE1CFFC
:10792000D9FFE2CFDAFFE652E652E652010EDF6EF1
:10793000D950FC0FE96EFF0EDA20EA6EEE50ED1022
:1079400030E0F80EDBCF3FF0F90EDBCF40F0DE5237
:107950003FC0DEFF40C0DDFFDD52D950010FE96EB0
:10796000000EDA20EA6EEE50ED1067E00001FD51E6
:10797000FE1163E0FC0EDBCFE9FFDB2AFD0EDBCF5F
:10798000EAFF01E3DB2AEF50E66EC7DCE5520001B7
:10799000FD07000EFE5B010EDB06020EDEE2DB06DB
:1079A000DCD7F80EDBCF00F0F90EDBCF01F0FA0EDA
:1079B000DBCF02F0FB0EDBCF03F000500110021012
:1079C00003103DE00001FCB712D0D950F80FE96E6A
:1079D000FF0EDA20EA6E090EE76ED890EF36010E40
:1079E000EB36020EEB36030EEB36E706F6E1D95026
:1079F000F80FE96EFF0EDA20EA6EEECFE6FFEECF6B
:107A0000E6FFEECFE6FFEFCFE6FF580EE66EA4DC12
:107A1000006E050EE15C02E2E16AE552E16E0050A3
:107A2000000957E1E66879DCE552FE0EE66E75DC8A
:107A3000E5520001FD6B020EFE6FDF6A4AD0020EB6
:107A40000001016AFD25006EFE510122010E00C0F9
:107A5000DBFF020E01C0DBFF010EDBCF00F0DB0617
:107A6000020EDBCF01F001E2DB060050011004E062
:107A7000E66A53DCE552F0D768DC1F0B050827E106
:107A8000880EF36E010EF3CFDBFF130EF36E020EC2
:107A9000F3CFDBFF5ADCFF0810E0D950010FE96E8D
:107AA000000EDA20EA6EEE50ED1007E013DC010E56
:107AB000DB06020EEFE2DB06EDD7D950010FE96ECF
:107AC000000EDA20EA6EEE50ED1001E0DF6A8280EF
:107AD0003CDCDF50E552E552E552E552E5CFDAFFF6
:067AE000E7CFD9FF120000
:0A7AE60081868A908A928A94938028
:107AF000938293849568938C938E9388938A9386CC
:107B000092900001AD6BAE6B1F6A206AFF0E1F5C86
:107B1000000E20580BE2000E1F24E96E010E2020FB
:107B2000EA6EEF6A1F2A000E2022F0D71F6A206A31
:107B3000FF0E1F5C000E20580BE2000E1F24E96EA2
:107B4000020E2020EA6EEF6A1F2A000E2022F0D7D4
:107B50002F6A1200D9CFE6FFDACFE6FFE1CFD9FFD7
:107B6000E2CFDAFF2C6A216A226A080E8A148A6E32
:107B700093868A908A928A948A9893809382938437
:107B800093889568630E2C5C01E1AAD08150400B6C
:107B900001E1A6D0A00E236E860E246E010E256E86
:107BA000266A2C50620A01E174D0640A62E0030A7A
:107BB00057E0010A4FE0070A45E0020A22E0030A03
:107BC00020E0020ADFE18150020B61E08150040BEA
:107BD0005EE023C000F024C001F025C002F026C002
:107BE00003F02306000E245A255A265AD880005442
:107BF000000E0154000E0254000E0354C3E3620E43
:107C00006DD0FC0EDBCF00F0FD0EDBCF01F00006E7
:107C1000000E015A0050211807E10150221804E11A
:107C2000020E1E1401E0939A000E2124E96E020E4A
:107C30002220EA6EEF1C8C6E212A000E2222956A09
:107C4000030E0AD081A202D0040E2C6EF2A49AD7A1
:107C5000040E0DD09390050E2C6ED66AF29492D736
:107C600081A402D0060E2C6EF2A48CD7060E2B6EC9
:107C700089D79568938A9380FC0EDBCF00F0FD0EC8
:107C8000DBCF01F00050215C0150225826E2010EAA
:107C900025D0820EE66E820EE66E880E006E820E93
:107CA000016E026A00C0E6FFE66E02C0E6FF800ECB
:107CB000E66E000EE66E7BEC43F0036E070EE15CB1
:107CC00002E2E16AE552E16E0350800EE66E000EBC
:107CD000E66EC7EC41F0E552E552630E2C6E52D7CA
:107CE0009380938293849388938A9568F70E931078
:107CF000936EE552E5CFDAFFE7CFD9FF1200D9CF77
:107D0000E6FFDACFE6FFE1CFD9FFE2CFDAFFE652B6
:107D1000E652DF6AD00E276E070E286E296A2A6A9D
:107D20000001AD6BAE6B010EDB6A8A6A93868A90A6
:107D30008A928A9481928194938093929394956885
:107D40002B6AE66AE66EE66A000EE66E010EE66EE5
:107D500038EC42F0006E050EE15C02E2E16AE552A9
:107D6000E16E0050630E2B5C01E1C5D00001000EF6
:107D7000AD5D010EAE5903E28150400B02E1090EE8
:107D80002B6E2B50090A01E1B1D0030A01E1AAD000
:107D90000C0A01E192D0030A45E0010A3FE0070A1C
:107DA00016E0010A0CE0030A05E0010ADBE1939208
:107DB000939481D09382D66AF294020E9AD081B0C5
:107DC00002D0030E2B6EF2A4CDD70A0E92D0D00EA5
:107DD000276E070E286E296A2A6A9392831CE66E24
:107DE000000EAD25E96E010EAE21EA6EE552E750B8
:107DF000EF6E8150200B01E0010E2D6E8150100BB3
:107E000001E0010E2E6EAD2B000EAE230A0E236E86
:107E1000246A256A266A9384040E6BD081A0A2D7B7
:107E2000050E67D093940F011F5118E02F50E66E96
:107E30002E5002E0000E01D0010EE66EADC0E9FF4B
:107E4000AEC0EAFFE906000EEA5A000EE926010E6E
:107E5000EA22EF50E66EC8EC19F017D02F50E66E0C
:107E60002E5002E0000E01D0010EE66EADC0E9FF1B
:107E7000AEC0EAFFE906000EEA5A000EE926010E3E
:107E8000EA22EF50E66EBFEC2CF0E552E552E552E7
:107E9000010EF3CFDBFFDB5027E12D500CE1060E86
:107EA0002B6EE80E236E030E246E256A266ADE52C0
:107EB000FE0EDD6E57D7010E1CD0938481AA02D02E
:107EC000090E2B6E2306000E245A255A265AD880F6
:107ED0002354000E2454000E2554000E265401E2B3
:107EE00041D702D0010EDF6E090E03D09392939416
:107EF000630E2B6E37D72E5030E1ADC0E9FFAEC018
:107F0000EAFFE906000EEA5A000EE926010EEA220F
:107F1000EF50600822E1ADC0E9FFAEC0EAFF020EFB
:107F2000E95E000EEA5A000EE926010EEA22EF5041
:107F30005F0813E1020E1E101E6EAFC000F2B0C04B
:107F400001F2020EE66EE66A05DEE552E552FD0E2E
:107F50001E141E6E0001AD6BAE6B0001000ED880CA
:107F6000AD55000EAE55DF5003E0F368F46A07D05C
:107F7000010EDB50006E016AF36E01C0F4FFE552A2
:107F8000E552E552E5CFDAFFE7CFD9FF1200819C39
:107F9000939CA00E236E860E246E010E256E266A1B
:107FA000235024102510261006E02306000E245A24
:107FB000255A265AF5D7818C938CA00E236E860EF7
:107FC000246E010E256E266A2350241025102610DB
:107FD00006E02306000E245A255A265AF5D7120029
:107FE000D9CFE6FFDACFE6FFE1CFD9FFE2CFDAFF64
:107FF000FD0EDB0403E19396819602D09386818681
:10800000E552E5CFDAFFE7CFD9FF1200D9CFE6FF7F
:10801000DACFE6FFE1CFD9FFE2CFDAFFE652E65250
:10802000D650026E036AD750046E056A3F6A010E8D
:10803000406E04C044F005C045F09AEC44F0025094
:108040003D24006E03503E2000C0DEFFDD6EF25086
:10805000040B01E0010EE66EE66ADECFE6FFDDCF3F
:10806000E6FFFD0EDBCF00F0016A00BE016800C034
:10807000E6FF01C0E6FF770E026E820E036E046A11
:1080800002C0E6FFE66E04C0E6FF800EE66E000E5C
:10809000E66E7BEC43F0056E0B0EE15C02E2E16AFA
:1080A000E552E16E0550800EE66E000EE66EC7ECFE
:1080B00041F0E552E552F294E552E552E552E5CF42
:0880C000DAFFE7CFD9FF12003F
:0880C8000D0A5469636B733A61
:1080D00025752025640D0A000D0A503A25642044B8
:1080E0003A25640044534B53454C004445425547A0
:1080F0000050524F544F000D0A4B3A257320563A08
:108100002573000D0A52656164202564206279742C
:108110006573000D0A52656164696E6720636F6E56
:10812000666967000D0A4D6F756E7420726574750F
:10813000726E73202558000D0A4D6F756E74696E4E
:1081400067002E00256300207C2000202530325857
:10815000000D0A000D0A44756D7020255820255821
:108160000D0A000D0A0D0A4F6F70732E204E6F20FE
:1081700063617264000D0A0D0A496E74657266616E
:10818000636520636C656172000D0A456467653A3A
:1081900020257320202564000D0A43617264206944
:1081A000732077726974652070726F74656374658B
:1081B00064000D0A4F70656E20257320726574751A
:1081C000726E73202558000D0A416D69676F203962
:1081D000313231440D0A000D0A53532F3830203903
:1081E0003133344C0D0A002F6C696664617461256B
:1081F000642E62696E000D0A0D0A53445F6D6F753F
:108200006E742072657475726E73202564000D0A99
:1082100048617264776172652050500D0A000D0A42
:10822000504F5254453A202558000D0A53544B5094
:1082300054523A202558000D0A53442053504920E7
:108240004449563A2025640031303A31363A3332C7
:10825000004D61722032352032303138000D0A2550
:1082600053202553000D0A0D0A48504469736B20B2
:108270007620302E3233000D0A25643A25752025EC
:1082800064007B4552527D002553000D0A436C6FFC
:1082900073696E67207772206661696C20256400BF
:1082A0000D0A5772697465206661696C2025640047
:1082B0000D0A5365656B20746F20256C6420666120
:1082C000696C6564202564000D0A72633D256400B5
:1082D0000D0A4D617820566563746F7220256C64B9
:0882E0002028256C582920001C
:0882E8000C0EAF6EB06AB896EF
:1082F000AC98AB8EAB88AB9A9D989D9AD08E9F8A96
:10830000F28EAC90AB9CAC9AAC8AAC940401819197
:10831000806B1200D9CFE6FFDACFE6FFE1CFD9FFBD
:10832000E2CFDAFFACA2FED7FD0EDBCFE6FFEBEC2F
:1083300044F0E552E552E5CFDAFFE7CFD9FF12006E
:108340009EBA03D0040007D8FBD7AE5000D012006D
:108350009EBA010C000CD9CFE6FFDACFE6FFE1CFE1
:10836000D9FFE2CFDAFFE652ABA204D0AC9AAC8AD6
:10837000AB98AB88ABA404D0AE50DF6EAC9AAC8A9D
:10838000E552E552E5CFDAFFE7CFD9FF1200D9CFAA
:10839000E6FFDACFE6FFE1CFD9FFE2CFDAFF040153
:1083A000826B836BFC0EDBCFE9FFFD0EDBCFEAFFB8
:1083B000EF5014E0FC0EDBCFE9FFFD0EDBCFEAFF50
:1083C000EF50E66EA7DFE552FC0EDB2AFD0E01E35F
:1083D000DB2A0401822B000E8323E4D7280E83AF0F
:1083E00002D0D89003D0825D000E835910E3230E93
:1083F000E66E90DFE5524F0EE66E8CDFE552460EDC
:10840000E66E88DFE552230EE66E84DFE552E55224
:0A841000E5CFDAFFE7CFD9FF120035
:06841A00D9CFE6FFDACF26
:10842000E6FFFA0EE3CFD9FFFB0EE3CFDAFFFC0E37
:10843000E3CFE9FFFD0EE3CFEAFFE9CFF3FFEACF99
:10844000F4FFF80EE35003E1F90EE35008E0F80EF4
:10845000E30602E2F90EE306DECFEEFFF2D7FF0EEF
:10846000E3CFDAFFE552FF0EE3CFD9FFE55212006A
:10847000FE0EE3CFE9FFFF0EE3CFEAFFE9CFF3FF04
:10848000EACFF4FFFB0EE35003E1FC0EE35009E0FA
:10849000FB0EE30602E2FC0EE306FD0EE350EE6E79
:1084A000F1D71200FD0EE3CFF6FFFE0EE3CFF7FF8C
:1084B000FF0EE3CFF8FFFB0EE3CFE9FFFC0EE3CFA7
:1084C000EAFFEE500900F55C02E1F566FAD712000A
:1084D000FE0EE3CFE9FFFF0EE3CFEAFFF36AF46A93
:1084E000EE5203E0F34AF42AFBD71200FF0EE3CF6B
:1084F000F8FFE552FF0EE3CFF7FFE552FF0EE3CFA3
:10850000F6FFE552E66AE66AE66A0900F55209E016
:10851000FD0EE32A05E1FE0EE32A02E1FF0EE32A47
:10852000F4D7FD0EE3CF3EF0FE0EE3CF3FF0FF0E9B
:06853000E3CF40F0120051
:0A853600FF0EE3CFEAFFE552FF0E4F
:10854000E3CFE9FFE552E66AE66AD9CFE6FFDACF84
:10855000E6FFFC0EE124D96EFF0EE220DA6EE66A39
:10856000E66AE66A200EEF5C06E0090EEF5C03E0C7
:10857000EF6603D03FD0EE50F5D72D0EEF5C03E150
:10858000FF0EE32A03D02B0EEF5C01E1EE502F0E1D
:10859000EF6424D03A0EEF6021D0D890F90EE33684
:1085A000FA0EE336FD0EDECFE3FFFE0EDDCFE3FF76
:1085B000D890F90EE336FA0EE336D890F90EE3368A
:1085C000FA0EE336FD0EE350DE26FE0EE350DD220A
:1085D000300EEE5CDE26000EDD22D9D7FF0EE3CF93
:1085E000E8FFE85207E0F90EE31EE32AFA0ED8B4DA
:1085F000E306E31EE552E552E552FF0EE3CFDAFF54
:10860000E552FF0EE3CFD9FFE552E1CFE9FFE2CF1C
:10861000EAFFED52ED52EECFF3FFEFCFF4FF120081
:10862000D9CFE6FFDACFE6FFE1CFD9FFE2CFDAFF1D
:10863000E652E652DE6ADD6ADECF00F0DDCF01F001
:10864000FC0EDBCF02F0FD0EDBCF03F00250005C2E
:10865000035001580AE2080EE66E14EC45F0E552AC
:10866000DF2A010EE9E3DB2AE7D7E552E552E552BE
:10867000E5CFDAFFE7CFD9FF1200D9CFE6FFDACF97
:10868000E6FFE1CFD9FFE2CFDAFFE652E652DE6A3B
:10869000DD6ADECF00F0DDCF01F0FC0EDBCF02F0B3
:1086A000FD0EDBCF03F00250005C035001580DE2D9
:1086B00000000000000000000000000000000000BA
:1086C000DF2A010E01E3DB2AE4D7E552E552E55249
:1086D000E5CFDAFFE7CFD9FF1200C2900F0EC16ECF
:1086E000070EB46ED36A4F0EC86E946A9488948253
:0686F0009484826A12006E
:0A86F600D9CFE6FFDACFE6FFE1CFAF
:10870000D9FFE2CFDAFFE652E652E652E652D950FE
:10871000F90F006EFF0EDA20016E020E00C0DBFFC3
:10872000030E01C0DBFF020EDBCFE6FF030EDBCF43
:10873000E6FFF90EDBCFE6FFFA0EDBCFE6FFFB0E1E
:10874000DBCFE6FFD950FC0FE66EFF0EDA20E66EB7
:1087500055EC33F0006E070EE15C02E2E16AE5528F
:10876000E16E0050F3CFDEFFF4CFDDFFFC0EDBCF78
:10877000E9FFFD0EDBCFEAFFEF6ADECF00F0DDCFD1
:1087800001F000C0F3FF01C0F4FF040EE15C02E25F
:10879000E16AE552E16EE552E5CFDAFFE7CFD9FFB6
:0287A0001200C5
:0E87A200060EF66E000EF76E000EF86E0F015A
:1087B0000900F5501A6F0900F5501B6F03E11A67A5
:1087C00001D03DD00900F550156F0900F550166F26
:1087D0000900F550176F09000900F550E96E09000E
:1087E000F550EA6E090009000900F550186F0900FC
:1087F000F550196F09000900F6CF1CFFF7CF1DFFD8
:10880000F8CF1EFF15CFF6FF16CFF7FF17CFF8FFF3
:108810000F01185302E1195307E00900F550EE6EFD
:108820001807F8E21907F9D71CCFF6FF1DCFF7FF9D
:108830001ECFF8FF0F011A07000E1B5BBFD71200F7
:10884000D9CFE6FFDACFE6FFE1CFD9FFE2CFDAFFFB
:10885000FB0EDBCF00F0FC0EDBCF01F00001800E41
:1088600001141AE1FB0EDBCFE9FFFC0EDBCFEAFFC0
:10887000EECFF3FFEDCFF4FFEE2A000EEF22F3CFA1
:10888000E9FFF4CFEAFFFD0EDBCFEFFFEF50016A07
:10889000F36E01C0F4FF10D0FB0EDB50FE0806E1C2
:1088A000FD0EDBCFE6FF42EC45F005D0FD0EDBCF41
:1088B000E6FF59EC45F0E552E552E5CFDAFFE7CFA8
:0488C000D9FF1200CA
:0C88C4003D504202F3CF39F0F4CF3AF0FF
:1088D0004302F3503A26000EF4203B6E3D50440212
:1088E000F3503B26000EF4203C6E3D504502F35001
:1088F0003C263E504202F3503A26F4503B22000EF2
:108900003C223E504302F3503B26F4503C223E5062
:108910004402F3503C263F504202F3503B26F450B1
:108920003C223F504302F3503C2640504202F35059
:048930003C261200CF
:0C89340040C04AF03FC049F03F504402F0
:10894000F4CF3EF0F3CF3DF040504502F4CF40F07D
:10895000F3CF3FF04402F3503E26F4503F22E86A42
:10896000402249504502F3503E26F4503F22E86A27
:10897000402245AEC0EF44F049503F5E4A50405A55
:0E8980004AAE000C44503F5E4550405A000C79
:02898E003C6A41
:108990003B6A3A6A396A200EE76ED8903D363E3619
:1089A0003F36403639363A363B363C364250395CF3
:1089B00043503A5844503B5845503C5809E34250C4
:1089C000395E43503A5A44503B5A45503C5A3D2A2E
:0689D000E72EE4D71200BF
:0A89D600D9CFE6FFDACFE6FFE1CFCC
:1089E000D9FFE2CFDAFFACAC04D0AC900001FFB30A
:1089F000AC80FD0EDB50AD6EE552E5CFDAFFE7CF80
:048A0000D9FF120088
:0C8A0400F36AF46AFF0EE124E96EFF0E35
:108A1000E220EA6EED6607D02F0EEF6404D03A0E26
:088A2000EF6001D0F32A1200FF
:088A2800FF0EE3504B6E480EF7
:108A300001D04C0EE76EE72EFED7E76AE72EFED791
:088A40004B2EF7D700001200D5
:088A4800800EF36E00EE00F059
:108A50000F0E01D81200EA6002D0EE6AFCD7F35084
:088A6000E9601200EE6AFCD788
:088A68001EEE00F02EEE00F0FE
:108A7000F86A389CD1EC43F05AEC45F07FEC23F0D7
:048A8000FBD712000E
:0C8A8400FF0EE350ACBA04D0AF6AAB8E1A
:108A9000AC8A949CACA2FED7AD6EF36EF46A120061
:108AA0003031323334353637383961626364656664
:018AB00000C5
:018AB100FFC5
:028AB2001200B0
:028AB4001200AE
:0A8AB6002F6C6966646174612E6222
:108AC000696E20002F68706469736B2E636667009F
:018AD00000A5
:0F8AD100800102E805000913400100010001F6D1
:108AE000008C119411941F01000000000000000090
:108AF000000000E34007000000003F005F0120018C
:0E8B00006501200040003400370000000A002C
:028B0E008000E5
:108B10004C4142454C310000000280000000000042
:108B2000000E00004D5946494C45313233340001A6
:108B300000000001000020001310120000000100DE
:088B400000000000000000002D
:020000040030CA
:0100010006F8
:0100020019E4
:010003001EDE
:010005008179
:010006008178
:00000001FF
